:020000020000FC
:100000000C9482311895189518951895189518958F
:100010001895189518951895189518951895189578
:100020001895189518951895189518951895189568
:100030001895189518951895189518951895189558
:100040001895189518951895189518951895189548
:100050000C948E0B18951895189518951895189559
:100060001895189518951895189518951895189528
:100070001895189518951895189518951895189518
:100080001895189518951895189518951895189508
:1000900018951895189518951895189518951895F8
:1000A00018951895189518951895189518951895E8
:1000B00018951895189518951895189518951895D8
:1000C00018951895189518951895189518951895C8
:1000D00018951895189518951895189518951895B8
:1000E00018951895189518951895189518951895A8
:1000F0001895189518951895189518951895189598
:100100001895189518951895189518951895189587
:100110001895189518951895189518950C947D0BA9
:100120001895189518951895189518951895189567
:10013000189518950C94E80A18951895189518951F
:100140001895189518951895189518951895189547
:100150001895189518951895189518951895189537
:100160001895189518951895189518951895189527
:100170001895189518951895189518951895189517
:100180001895189518951895189518951895189507
:1001900018951895189518951895189518951895F7
:1001A00018951895189518951895189518951895E7
:1001B00018951895189518951895189518951895D7
:1001C00018951895189518951895189518951895C7
:1001D00018951895189518951895189518951895B7
:1001E00018951895189518951895189518951895A7
:1001F00018951895189518951895189544241FBCAE
:1002000037CB7ABC26B8A2BD41F61CBE6EBA0DBE75
:10021000FC0C633C5C1D633E6EE3A33E5C1D633ED1
:10022000FC0C633C6EBA0DBE41F61CBE26B8A2BDE6
:1002300037CB7ABC44241FBC631349BEDBD713BE43
:100240003B43DA3BD34F453EE0C1903ED34F453E62
:100250003B43DA3BDBD713BE631349BE14BEA1BDDB
:100260006FEDFCBDDC252FBEE9383F3FDC252FBEFE
:100270006FEDFCBD14BEA1BD90F90F3F90F90FBF0B
:100280000000803FFE98FFBDE5FF3CBE6A8B31BE9B
:10029000D6704CBC0186593E0595A33E0186593E59
:1002A000D6704CBC6A8B31BEE5FF3CBE1F1F1F00E1
:1002B000000000001C1E1F1F1F1F1F1F1F1F1F1FCE
:1002C0001F1F1E1C00000000001F1F1F1F1F1F1FDD
:1002D0001F1F0F07070F1F1F1F1F1F1F00000000FA
:1002E000001F1F1F1F1F1F00001F1F1F05000104ED
:1002F00003022020052020FF000701040306000759
:10030000010603020506FF2020FF05070006030281
:100310000507000403020000012020FF0507010477
:100320000302050701030302050707042020050750
:1003300007040303050701042020001F2C3D630070
:100340000102040810204000000000010101012406
:10035000212A21302136213A213D214121452149BF
:10036000214D21522157215C212A2A2A2A2A2A2A70
:100370002A2A00004628100045221824D3241B25D1
:100380004D259225C22507264C269226CD26FD26F0
:1003900040279027CE270A280000C62C10002129CC
:1003A000C62C6F2AC62C8A2AD42AD82BFA2B122CB8
:1003B000C62C00313E2C572C6F2CC62C872C0000ED
:1003C000E92E1000DC2C1B2D2E2D432D622D8D2DA2
:1003D000B82DD22DE72D5A2E6B2E922EA32EB42E91
:1003E000C52EDC2E0000F9301000FF2E432F562FB3
:1003F0006B2F842FAF2FD82FF22F07306C307D302A
:10040000A230B330C430D530EC3000014F374C3718
:10041000453F37023F3711A9360B6E3601C736010B
:100420003F37013F37013F3702C736055B36019C36
:100430003601A93603773602A93603A536FB00E359
:1004400030D000E815E237D100E815E234D100E8F9
:1004500015E231D100E325D000E815E22CD100E30C
:1004600020D000EC13E027D102E01BD000EC13E019
:1004700022D108E016D000EC13E01DD101E011D02C
:1004800000E815E218D100E815E215D106E009D020
:1004900000EC13E010D10CE004D000EC13E00BD121
:1004A00008958A93802FE4E4F6E000810F7B0083B7
:1004B00000E310E000D100916406007F0093640621
:1004C000082F02950F7010916406102B109364068C
:1004D000E4E4F6E000810068008300E310E0EBD084
:1004E000E4E4F6E000810F77008300EF10E0E3D052
:1004F00000916406007F009364068F70009164068B
:10050000082B00936406E4E4F6E0008100680083B1
:1005100000E310E0D0D0E4E4F6E000810F77008340
:1005200000EF10E0C8D0899108958A93802FE4E409
:10053000F6E000810064008300E310E0BCD000918D
:100540006406007F00936406082F02950F701091D7
:100550006406102B10936406E4E4F6E00081006862
:10056000008300E310E0A7D0E4E4F6E000810F7719
:10057000008300EF10E09FD000916406007F00939D
:1005800064068F7000916406082B00936406E4E40F
:10059000F6E000810068008300E310E08CD0E4E422
:1005A000F6E000810F77008300EF10E084D089919E
:1005B00008950E940735C801A0E007C0B0E0FC0123
:1005C000EA0FFB1F0081B1DFA395B0E0FC01EA0F49
:1005D000FB1F0081002311F0A13180F3E4E00C94B3
:1005E00018355FDF0FE915E2E4DF08951BEC109387
:1005F000520018E010935000E1E5F0E0108113FF85
:10060000FBCF003221F402EC0093550003C003EC51
:1006100000935500E0E5F0E0008100610083E1E532
:10062000F0E0008104FFFBCF08ED04BF04E000937D
:100630004000E0E5F0E000810E7F0083089504E4CF
:1006400014E000930C0210930D0200E100930102EC
:1006500002E20093020203E00093040203E000932D
:10066000200208E200932102E0E0F2E00081016054
:100670000083089501E00093280200E3009329021B
:10068000089501E00093300208E3009331020895D9
:100690000DE00093200300E40093210300E00093A9
:1006A000220300E50093240300E70093280300EEF3
:1006B00000932A0308950150104098018901232BCB
:1006C000D1F708958A93802F04C008EE1DEF0E9491
:1006D00034118A95082F802F0023B9F78991089546
:1006E0000E94063580E090E0A0E0B0E04EE0442EAD
:1006F0001BC0442D50E0440F551F440F551FFA01F5
:10070000E555FA4D0080118022803380442D50E061
:10071000440F551F440F551FFA01E155FA4D008251
:100720001182228233824A9441E0441610F7EFEAA4
:10073000F5E20083118322833383442423C0042DF4
:1007400010E0000F111F000F111FF801E450FE4FC1
:100750004591559165917491042D10E0000F111F82
:10076000000F111FF801E155FA4D0081118122811E
:1007700033810E948B33AC01BD010E942A33C80132
:10078000D90143940FE04016D0F28C019D01E5E0C1
:100790000C9417350E94063580E090E0A0E0B0E0B0
:1007A0004EE0442E1BC0442D50E0440F551F440F13
:1007B000551FFA01E951FA4D0080118022803380E3
:1007C000442D50E0440F551F440F551FFA01E551C9
:1007D000FA4D00821182228233824A9441E044160B
:1007E00010F7EBEEF5E20083118322833383442478
:1007F00023C0042D10E0000F111F000F111FF8017E
:10080000E450FE4F4591559165917491042D10E08F
:10081000000F111F000F111FF801E551FA4D008163
:100820001181228133810E948B33AC01BD010E9472
:100830002A33C801D90143940FE04016D0F28C014D
:100840009D01E5E00C9417350E94063580E090E0AC
:10085000A0E0B0E04EE0442E1BC0442D50E0440F19
:10086000551F440F551FFA01ED5DF94D00801180B1
:1008700022803380442D50E0440F551F440F551FF4
:10088000FA01E95DF94D00821182228233824A9495
:1008900041E0441610F7E7E2F6E200831183228379
:1008A0003383442423C0042D10E0000F111F000FD8
:1008B000111FF801E450FE4F4591559165917491D7
:1008C000042D10E0000F111F000F111FF801E95D4A
:1008D000F94D00811181228133810E948B33AC015B
:1008E000BD010E942A33C801D90143940FE040168C
:1008F000D0F28C019D01E5E00C9417350E9406357D
:1009000080E090E0A0E0B0E048E0442E1BC0442D21
:1009100050E0440F551F440F551FFA01E15AF94D9D
:100920000080118022803380442D50E0440F551FF9
:10093000440F551FFA01ED59F94D008211822282B0
:1009400033824A9441E0441610F7E3E6F6E200836E
:10095000118322833383442423C0042D10E0000F2D
:10096000111F000F111FF801E85CFD4F45915591D3
:1009700065917491042D10E0000F111F000F111FDD
:10098000F801ED59F94D00811181228133810E94D6
:100990008B33AC01BD010E942A33C801D9014394B5
:1009A00009E04016D0F28C019D01E5E00C9417356A
:1009B0000E94063580E090E0A0E0B0E048E0442EE0
:1009C0001BC0442D50E0440F551F440F551FFA0122
:1009D000ED57F94D0080118022803380442D50E086
:1009E000440F551F440F551FFA01E957F94D008276
:1009F0001182228233824A9441E0441610F7E7E8DC
:100A0000F6E20083118322833383442423C0042D20
:100A100010E0000F111F000F111FF801E85CFD4FDF
:100A20004591559165917491042D10E0000F111FAF
:100A3000000F111FF801E957F94D00811181228142
:100A400033810E948B33AC01BD010E942A33C8015F
:100A5000D901439409E04016D0F28C019D01E5E0F4
:100A60000C9417350E94063580E090E0A0E0B0E0DD
:100A700048E0442E1BC0442D50E0440F551F440F46
:100A8000551FFA01E955F94D00801180228033800D
:100A9000442D50E0440F551F440F551FFA01E555F2
:100AA000F94D00821182228233824A9441E0441639
:100AB00010F7EBEAF6E200831183228333834424A8
:100AC00023C0042D10E0000F111F000F111FF801AB
:100AD000E85CFD4F4591559165917491042D10E0AE
:100AE000000F111F000F111FF801E555F94D00818E
:100AF0001181228133810E948B33AC01BD010E94A0
:100B00002A33C801D901439409E04016D0F28C0180
:100B10009D01E5E00C9417350E94063580E090E0D9
:100B2000A0E0B0E046E0442E1BC0442D50E0440F4E
:100B3000551F440F551FFA01E553F94D00801180F0
:100B400022803380442D50E0440F551F440F551F21
:100B5000FA01E153F94D00821182228233824A94D4
:100B600041E0441610F7EFECF6E200831183228394
:100B70003383442423C0042D10E0000F111F000F05
:100B8000111FF801E45AFD4F4591559165917491FB
:100B9000042D10E0000F111F000F111FF801E15389
:100BA000F94D00811181228133810E948B33AC0188
:100BB000BD010E942A33C801D901439407E04016C1
:100BC000D0F28C019D01E5E00C9417350E940635AA
:100BD00080E090E0A0E0B0E046E0442E1BC0442D51
:100BE00050E0440F551F440F551FFA01E951F94DCC
:100BF0000080118022803380442D50E0440F551F27
:100C0000440F551FFA01E551F94D008211822282ED
:100C100033824A9441E0441610F7EBEEF6E200838B
:100C2000118322833383442423C0042D10E0000F5A
:100C3000111F000F111FF801E45AFD4F4591559106
:100C400065917491042D10E0000F111F000F111F0A
:100C5000F801E551F94D00811181228133810E9413
:100C60008B33AC01BD010E942A33C801D9014394E2
:100C700007E04016D0F28C019D01E5E00C94173599
:100C80000E94063580E090E0A0E0B0E046E0442E0F
:100C90001BC0442D50E0440F551F440F551FFA014F
:100CA000ED5FF84D0080118022803380442D50E0AC
:100CB000440F551F440F551FFA01E95FF84D00829C
:100CC0001182228233824A9441E0441610F7E7E011
:100CD000F7E20083118322833383442423C0042D4D
:100CE00010E0000F111F000F111FF801E45AFD4F13
:100CF0004591559165917491042D10E0000F111FDD
:100D0000000F111FF801E95FF84D00811181228168
:100D100033810E948B33AC01BD010E942A33C8018C
:100D2000D901439407E04016D0F28C019D01E5E023
:100D30000C9417350E94033581E035C0482F50E0F0
:100D4000440F551F440F551FFA01E95DF84D00800F
:100D5000118022803380482F50E0440F551F440FEC
:100D6000551FFA01E55DF84D00821182228233821F
:100D7000482F50E0440F551F440F551FFA01E15E04
:100D8000F84D0080118022803380482F50E0440FBE
:100D9000551F440F551FFA01ED5DF84D0082118279
:100DA000228233828A95813048F6EBE2F7E20083B3
:100DB000118322833383EBE2F7E240815181628128
:100DC0007381E8E7F2E005911591259134910E9435
:100DD0008B33E3E2F7E2008311832283338381E0E4
:100DE0004FC0082F10E0000F111F000F111FF80156
:100DF000E858FD4F4591559165917491082F10E089
:100E0000000F111F000F111FF801E55DF84D008163
:100E10001181228133810E948B3328013901082FEF
:100E200010E0000F111F000F111FF801E058FD4FD7
:100E30004591559165917491082F10E0000F111F95
:100E4000000F111FF801ED5DF84D00811181228125
:100E500033810E948B33A801B901820193010E9462
:100E60006E33E3E2F7E240815181628173810E9437
:100E70002A33E3E2F7E200831183228333838395ED
:100E8000823008F4AECFE3E2F7E2008111812281E3
:100E90003381E8E00C9414350E94033581E035C0BD
:100EA000482F50E0440F551F440F551FFA01E95CCD
:100EB000F84D0080118022803380482F50E0440F8D
:100EC000551F440F551FFA01E55CF84D0082118251
:100ED00022823382482F50E0440F551F440F551F84
:100EE000FA01E15DF84D0080118022803380482FA7
:100EF00050E0440F551F440F551FFA01ED5CF84DAB
:100F000000821182228233828A95813048F6EBE397
:100F1000F7E20083118322833383EBE3F7E240811E
:100F2000518162817381E8E7F2E005911591259185
:100F300034910E948B33E3E3F7E200831183228331
:100F4000338381E04FC0082F10E0000F111F000F06
:100F5000111FF801E858FD4F459155916591749125
:100F6000082F10E0000F111F000F111FF801E55CA2
:100F7000F84D00811181228133810E948B33280139
:100F80003901082F10E0000F111F000F111FF80189
:100F9000E058FD4F4591559165917491082F10E0EF
:100FA000000F111F000F111FF801ED5CF84D0081BB
:100FB0001181228133810E948B33A801B901820102
:100FC00093010E946E33E3E3F7E240815181628135
:100FD00073810E942A33E3E3F7E2008311832283C3
:100FE00033838395823008F4AECFE3E3F7E20081E8
:100FF000118122813381E8E00C9414350E9403357D
:1010000081E035C0482F50E0440F551F440F551F55
:10101000FA01E95BF84D0080118022803380482F6F
:1010200050E0440F551F440F551FFA01E55BF84D82
:101030000082118222823382482F50E0440F551FD4
:10104000440F551FFA01E15CF84D008011802280A9
:101050003380482F50E0440F551F440F551FFA01AD
:10106000ED5BF84D00821182228233828A958130B5
:1010700048F6EBE4F7E20083118322833383EBE449
:10108000F7E24081518162817381E8E7F2E00591E6
:101090001591259134910E948B33E3E4F7E20083AC
:1010A00011832283338381E04FC0082F10E0000FAB
:1010B000111F000F111FF801E858FD4F4591559180
:1010C00065917491082F10E0000F111F000F111F80
:1010D000F801E55BF84D00811181228133810E9486
:1010E0008B3328013901082F10E0000F111F000F6A
:1010F000111FF801E058FD4F45915591659174918C
:10110000082F10E0000F111F000F111FF801ED5BF9
:10111000F84D00811181228133810E948B33A80117
:10112000B901820193010E946E33E3E4F7E240814A
:101130005181628173810E942A33E3E4F7E20083E4
:101140001183228333838395823008F4AECFE3E4A6
:10115000F7E20081118122813381E8E00C9414359B
:101160000E940335842FA52F0E94CB32482F50E0D8
:10117000440F551F440F551FFA01ED5AF84D408199
:101180005181628173810E946E33280139010A2FD7
:1011900010E020E030E00E94D632A801B9018201BF
:1011A00093010E940434482F50E0440F551F440F10
:1011B000551FFA01ED5AF84D4081518162817381CA
:1011C0000E942A3390E0880F991F880F991FFC0115
:1011D000ED5AF84D0083118322833383E8E00C94A9
:1011E00014350E94063580E090E0A0E0B0E048E0D1
:1011F000442E1BC0442D50E0440F551F440F551F73
:10120000FA01E157F84D0080118022803380442D8F
:1012100050E0440F551F440F551FFA01ED56F84D8D
:1012200000821182228233824A9441E0441610F7F0
:10123000E3E9F7E20083118322833383442423C04C
:10124000042D10E0000F111F000F111FF801E857C7
:10125000FD4F4591559165917491042D10E0000F5B
:10126000111F000F111FF801ED56F84D008111817B
:10127000228133810E948B33AC01BD010E942A334D
:10128000C801D901439409E04016D0F28C019D01B8
:10129000E5E00C9417350E94063580E090E0A0E070
:1012A000B0E048E0442E1BC0442D50E0440F551FD1
:1012B000440F551FFA01ED54F84D00801180228033
:1012C0003380442D50E0440F551F440F551FFA0141
:1012D000E954F84D00821182228233824A9441E01F
:1012E000441610F7E7EBF7E2008311832283338380
:1012F000442423C0042D10E0000F111F000F111F04
:10130000F801E857FD4F4591559165917491042D71
:1013100010E0000F111F000F111FF801E954F84DE4
:1013200000811181228133810E948B33AC01BD0188
:101330000E942A33C801D901439409E04016D0F233
:101340008C019D01E5E00C9417350E94063580E084
:1013500090E0A0E0B0E048E0442E1BC0442D50E0F7
:10136000440F551F440F551FFA01E952F84D0080F4
:10137000118022803380442D50E0440F551F440FCC
:10138000551FFA01E552F84D008211822282338204
:101390004A9441E0441610F7EBEDF7E20083118325
:1013A00022833383442423C0042D10E0000F111F37
:1013B000000F111FF801E857FD4F459155916591B8
:1013C0007491042D10E0000F111F000F111FF80180
:1013D000E552F84D00811181228133810E948B33C7
:1013E000AC01BD010E942A33C801D901439409E030
:1013F0004016D0F28C019D01E5E00C941735109158
:10140000480001E0009348002091A0003091A20024
:101410000091A2000C7F04600093A2004FB7789463
:10142000E8E4F0E00081016000835091CD01EF938A
:10143000FF930F932F93EBECF1E008ED21E004BF55
:1014400020832F910F91FF91EF9103E00093CD0145
:101450008895109348002093A0003093A2005093E9
:10146000CD014FBF0895EFECF1E0008107FDFBCF08
:101470000895F9DFEFECF1E0008101FF11C006E310
:101480000093CA01EF93FF930F932F93EBECF1E0DE
:1014900008ED21E004BF20832F910F91FF91EF9180
:1014A00008959A938A93C801DEDFFC01E05CF14065
:1014B000F09750F44091A82950E009E010E00E9414
:1014C000D031800F911F17C0803C01E0900798F445
:1014D0004091A72950E00BE110E00E94D031980123
:1014E0004091A82950E001E510E00E94D031200F82
:1014F000311F820F931F082F0093C001892F8F7116
:101500008093C10100E00093C20106E00093CA018C
:10151000EF93FF930F932F93EBECF1E008ED21E0B5
:1015200004BF20832F910F91FF91EF910091C4018F
:101530008991999108950E940835C801A22F00E071
:101540000093060900E000934608FC01E05CF140CE
:10155000F09750F44091A82950E009E010E00E9473
:10156000D031800F911F17C0803C01E0900798F4A4
:101570004091A72950E00BE110E00E94D031980182
:101580004091A82950E001E510E00E94D031200FE1
:10159000311F820F931F6DDF03E30093CA01082FF1
:1015A0000093C001892F8F718093C10100E00093E7
:1015B000C201A093C40105E30093CA0120DF03E048
:1015C0000093060901E000934608E3E00C94193506
:1015D0009A938A93FA93EA932A921A920A927A93A6
:1015E0006A935A934A933A932A931A930A932FB67B
:1015F000E0E0F2E00081046000830091722903952D
:101600000770009372290091722910E0F801E95BDC
:10161000FC4F0491002339F404E00093450608E0F0
:101620000093460606C004E00093460608E00093D7
:1016300045064091932950E006E212E00E94D03125
:1016400000933A0310933B030091722910E0000FBE
:10165000111FF801E150F84D00811181009338030A
:1016600010933903009175290023B1F10091BF282F
:101670001091C028212F220F220B322F4091722966
:1016800050E0440F551F440F551FFA01E158F74D24
:101690004081518162817381400F511F621F731F0E
:1016A00040835183628373838091D3289091D4289F
:1016B00001968093D3289093D4280091D528109137
:1016C000D6288017910741F400E00093752910E0B7
:1016D0000093D3281093D4282FBE099119912991F2
:1016E000399149915991699179910990199029906D
:1016F000E991F9918991999118952A931A930A93EE
:101700002FB700911002109111020093BF2810937F
:10171000C0282FBF09911991299118955A924A9280
:10172000BA93AA939A938A93FA93EA933A922A9253
:101730001A920A927A936A935A934A933A932A9303
:101740001A930A935FB600917529002309F076C5B4
:1017500000919929002309F100919929102F1A95D8
:1017600010939929002339F400E00093992900E0AF
:101770000093400912C000918D2910919A29019F70
:101780004091992950E080010E94D03143E00E94AD
:10179000E43100936A0910936B09009183290E5F6D
:1017A0000093912980E037C050919129482F642FF0
:1017B000082F10E0000F111F000F111FF801E15852
:1017C000F74D008111812281338142E00E943E3237
:1017D000462FC6DC0E94D832482F50E0440F551FD8
:1017E000440F551FFA01E156F74D00831183228300
:1017F000338300E010E020E030E0482F50E0440F59
:10180000551F440F551FFA01E158F74D008311830E
:10181000228333838395883038F20FEF0093752944
:1018200000E010E020E030E0E7EEF8E20083118312
:1018300022833383E3EEF8E2008311832283338330
:10184000EFEDF8E2008311832283338300E010E0A0
:1018500020E030E0E3EAF9E200831183228333835E
:101860004424C9C0042D10E0000F111F000F111FE8
:10187000F801E156F74D4081518162817381042D59
:1018800010E0000F111F000F111FF801E156F74D76
:1018900000811181228133810E9416320E94CB3255
:1018A000E3EAF9E240815181628173810E942A3327
:1018B000E3EAF9E20083118322833383EFEDF8E258
:1018C00000811181228133810E94CB32C801D9016C
:1018D000042D10E0000F111F000F111FF801E15639
:1018E000F74D00811181228133810E94CB32442D3A
:1018F00050E0440F551F440F551FFA01E15EF74DAC
:1019000040815181628173810E948B33AC01BD01A2
:101910000E942A330E94D832EFEDF8E2008311834F
:1019200022833383E3EEF8E2008111812281338147
:101930000E94CB32C801D901042D10E0000F111F05
:10194000000F111FF801E156F74D0081118122812E
:1019500033810E94CB32442D50E0440F551F440F79
:10196000551FFA01E15CF74D40815181628173811D
:101970000E948B33AC01BD010E942A330E94D832F1
:10198000E3EEF8E20083118322833383E7EEF8E28B
:1019900000811181228133810E94CB32C801D9019B
:1019A000042D10E0000F111F000F111FF801E15668
:1019B000F74D00811181228133810E94CB32442D69
:1019C00050E0440F551F440F551FFA01E15AF74DDF
:1019D00040815181628173810E948B33AC01BD01D2
:1019E0000E942A330E94D832E7EEF8E20083118386
:1019F00022833383439408E0401608F433CF40E059
:101A000050E060E071E4E3EAF9E2008111812281B3
:101A100033810E9404340E946F39E3EAF9E20083C3
:101A200011832283338300919529013099F4E3EAED
:101A3000F9E200811181228133810E94D8324091E4
:101A4000D9285091DA280E94EA310093D1281093C6
:101A5000D22814C0E3EAF9E20081118122813381A6
:101A60000E94D8324091D9285091DA28440F551F4E
:101A70000E94EA310093D1281093D2280091922934
:101A800010E0F801E15CFC4F449150E00091D12856
:101A90001091D2280E94EA310093D1281093D228C5
:101AA00000919629023051F40091D1281091D2284A
:101AB000169507950093D1281093D228EFEDF8E200
:101AC0000081118122813381E3EFF8E200831183E9
:101AD00022833383E3EEF8E2008111812281338196
:101AE000E7EFF8E20083118322833383E7EEF8E225
:101AF0000081118122813381EFEFF8E200831183AD
:101B000022833383EBE0F9E200811181228133816A
:101B1000EFEFF8E24081518162817381041715076C
:101B2000260737077CF4EBE0F9E20081118122817E
:101B300033810F5F1F4F2F4F3F4F0083118322834D
:101B400033830EC0EBE0F9E2008111812281338101
:101B500001501040204030400083118322833383A2
:101B6000E7E0F9E20081118122813381E3EFF8E2BD
:101B70004081518162817381041715072607370759
:101B80007CF4E7E0F9E200811181228133810F5F6B
:101B90001F4F2F4F3F4F00831183228333830EC08B
:101BA000E7E0F9E200811181228133810150104088
:101BB000204030400083118322833383E3E0F9E245
:101BC0000081118122813381E7EFF8E24081518168
:101BD0006281738104171507260737077CF4E3E059
:101BE000F9E200811181228133810F5F1F4F2F4F56
:101BF0003F4F00831183228333830EC0E3E0F9E279
:101C000000811181228133810150104020403040F9
:101C1000008311832283338300917429002339F1D7
:101C200000E000937429E3EFF8E200811181228142
:101C30003381E7E0F9E20083118322833383E7EF06
:101C4000F8E20081118122813381E3E0F9E200832F
:101C5000118322833383EFEFF8E200811181228127
:101C60003381EBE0F9E20083118322833383E7E0E1
:101C7000F9E20081118122813381E3EFF8E24081B2
:101C8000518162817381401B510B620B730B408346
:101C9000518362837383E3E0F9E200811181228141
:101CA0003381E7EFF8E24081518162817381401B0B
:101CB000510B620B730B4083518362837383EBE0A0
:101CC000F9E20081118122813381EFEFF8E2408156
:101CD000518162817381401B510B620B730B4083F6
:101CE0005183628373830091DD281091DE280130D7
:101CF00020E0120709F021C100919529023009F472
:101D0000E8C000918F290130B9F5E3EFF8E20081D6
:101D10001181228133810E94CB320E9470030E9484
:101D2000D832EBE2F9E20083118322833383E7EFB9
:101D3000F8E200811181228133810E94CB320E941E
:101D4000CA030E94D832EFE2F9E2008311832283B2
:101D50003383EFEFF8E200811181228133810E9409
:101D6000CB320E9424040E94D832E7E2F9E20083D9
:101D700011832283338305C100918F290230B9F585
:101D8000E3EFF8E200811181228133810E94CB329E
:101D90000E947E040E94D832EBE2F9E200831183B4
:101DA00022833383E7EFF8E20081118122813381BE
:101DB0000E94CB320E94D8040E94D832EFE2F9E2AE
:101DC0000083118322833383EFEFF8E200811181D6
:101DD000228133810E94CB320E9432050E94D83288
:101DE000E7E2F9E20083118322833383CAC00091C2
:101DF0008F290330B9F5E3EFF8E2008111812281E8
:101E000033810E94CB320E948C050E94D832EBE2D3
:101E1000F9E20083118322833383E7EFF8E2008144
:101E20001181228133810E94CB320E94E6050E94FB
:101E3000D832EFE2F9E20083118322833383EFEF9C
:101E4000F8E200811181228133810E94CB320E940D
:101E500040060E94D832E7E2F9E200831183228330
:101E600033838FC0E3EFF8E2008111812281338157
:101E70000E94CB320E949A060E94D832EBE2F9E22D
:101E80000083118322833383E7EFF8E2008111811D
:101E9000228133810E94CB320E944C070E94D832AB
:101EA000EFE2F9E20083118322833383EFEFF8E25C
:101EB00000811181228133810E94CB320E94FE0772
:101EC0000E94D832E7E2F9E2008311832283338350
:101ED00058C0E3EFF8E200811181228133810E9432
:101EE000CB327FD90E94D832EBE2F9E20083118332
:101EF00022833383E7EFF8E200811181228133816D
:101F00000E94CB32C8D90E94D832EFE2F9E20083B6
:101F1000118322833383EFEFF8E200811181228164
:101F200033810E94CB3211DA0E94D832E7E2F9E223
:101F3000008311832283338324C0E3EFF8E200811E
:101F4000118122813381EBE2F9E200831183228344
:101F50003383E7EFF8E20081118122813381EFE2E0
:101F6000F9E20083118322833383EFEFF8E20081EB
:101F7000118122813381E7E2F9E200831183228318
:101F8000338300918A29009500938A2900918A2938
:101F9000002309F023C1EBE2F9E2008111812281E3
:101FA0003381E7E3F9E24081518162817381040F5B
:101FB000151F261F371FE3E4F9E2008311832283F4
:101FC0003383EFE2F9E20081118122813381EBE377
:101FD000F9E24081518162817381040F151F261F30
:101FE000371FE7E4F9E20083118322833383E7E2BA
:101FF000F9E20081118122813381E3E3F9E240813A
:10200000518162817381040F151F261F371FEFE373
:10201000F9E20083118322833383EFEFF8E200813A
:10202000118122813381EBE5F9E2408151816281A6
:102030007381040F151F261F371FEFE5F9E2008398
:1020400011832283338300918B29009500938B2980
:1020500000918B29002309F090C0E3E4F9E20081AC
:10206000118122813381EBE4F9E240815181628167
:102070007381040F151F261F371F43E050E0609146
:10208000962970E0461B570B652F660F660B762F5F
:102090000E946932EBEEF8E20083118322833383DE
:1020A000E7E4F9E20081118122813381EFE4F9E272
:1020B0004081518162817381040F151F261F371FD4
:1020C00043E050E06091962970E0461B570B652F66
:1020D000660F660B762F0E946932EFEEF8E20083FE
:1020E000118322833383EFE3F9E20081118122819E
:1020F0003381E3E5F9E24081518162817381040F0C
:10210000151F261F371F43E050E06091962970E0AD
:10211000461B570B652F660F660B762F0E946932A0
:10212000EBEFF8E20083118322833383EFE5F9E2DA
:102130000081118122813381E3E6F9E240815181FE
:1021400062817381040F151F261F371F43E050E083
:102150006091962970E0461B570B652F660F660B42
:10216000762F0E946932E7E5F9E20083118322832A
:1021700033830FEF00938C2961C0E3E4F9E200811F
:10218000118122813381EBE4F9E200831183228300
:102190003383E7E4F9E20081118122813381EFE4A6
:1021A000F9E20083118322833383EFE3F9E20081B4
:1021B000118122813381E3E5F9E2008311832283D7
:1021C0003383EFE5F9E20081118122813381E3E677
:1021D000F9E2008311832283338330C0EBE2F9E21A
:1021E0000081118122813381E7E3F9E200831183C9
:1021F00022833383EFE2F9E200811181228133816E
:10220000EBE3F9E20083118322833383E7E2F9E20F
:102210000081118122813381E3E3F9E2008311839C
:1022200022833383EFEFF8E2008111812281338131
:10223000EBE5F9E200831183228333835FBE0991CA
:1022400019912991399149915991699179910990FF
:10225000199029903990E991F99189919991A991D1
:10226000B9914990599018959C01C8010197FC01BA
:10227000CF01EF2BD9F716950795C8010197FC01FF
:10228000CF01EF2BD9F7C90108950E94073500E46B
:102290000E945102AFEF80E002C0A695839588307E
:1022A000A8F4BA2F90E005C000E00E949502B69510
:1022B0009395983090F7BB2311F001E001C000E046
:1022C000002391F70FE10E949502F1CFE4E00C9416
:1022D00018359A938A9300E40E94510280E008C066
:1022E00090E0FC01E455FD4F04910E949502839516
:1022F0008034B0F38991999108950E940735D801EF
:1023000080E090E02AC00DE210E0AC010E94D031E4
:10231000F801EA0FFB1FE83601E0F00714F0E85679
:10232000F1408F01212F220F220B322F0E94CB323E
:1023300045E35AEF6EE87CE30E948B330E947E31C6
:10234000AC01440F551F440F551FFA01E15AF74DD8
:1023500000831183228333830196883000E0900745
:1023600094F2E4E00C9418350E940735D80180E01F
:1023700090E02AC00DE210E0AC010E94D031F801DB
:10238000EA0FFB1FE83601E0F00714F0E856F140D1
:102390008F01212F220F220B322F0E94CB3245E3D7
:1023A0005AEF6EE87CE30E948B330E94A138AC01A7
:1023B000440F551F440F551FFA01E15EF74D00838E
:1023C0001183228333830196883000E0900794F2D2
:1023D000E4E00C9418350E940735D80180E090E0C5
:1023E0002AC00DE210E0AC010E94D031F801EA0FE2
:1023F000FB1FE83601E0F00714F0E856F1408F01CA
:10240000212F220F220B322F0E94CB3245E35AEFAD
:102410006EE87CE30E948B330E947E31AC01440F56
:10242000551F440F551FFA01E15CF74D00831183DE
:10243000228333830196883000E0900794F2E4E031
:102440000C9418350E940335D80180E090E013C049
:10245000FC01E95BFC4F049110E0AD010E94D0311A
:10246000000F111F9C01220F331FF901E15FF74D8F
:10247000008311830196883000E090070CF046C07D
:1024800000917B29002321F70DE210E0AC010E94AE
:10249000D031A80146535F4F483601E0500714F091
:1024A000485651408D01212F220F220B322F0E94BE
:1024B000CB32280139018A01212F220F220B322F22
:1024C0000E94CB3245E35AEF6EE87CE30E948B33E7
:1024D0000E94A138A201B3010E948B332801390167
:1024E0008D01212F220F220B322F0E94CB32A2010D
:1024F000B3010E942A330E94D8329C01220F331F5D
:10250000F901E15FF74D00831183B4CFE8E00C944B
:1025100014350E9401354801D90180E090E046C0A1
:102520000DE210E0AC010E94D031A801480D591D08
:10253000483601E0500714F0485651408D01212FD4
:10254000220F220B322F0E94CB32280139018A013F
:10255000212F220F220B322F0E94CB3208011901AA
:1025600045E35AEF6EE87CE3800191010E948B33D2
:102570000E94A138A201B3010E948B3328013901C6
:102580008D01212F220F220B322F0E94CB32A2016C
:10259000B3010E942A330E94D8329C01220F331FBC
:1025A000F901E150F84D008311830196883000E075
:1025B00090070CF4B5CFEAE00C9412350E94073571
:1025C00020E030E000E010E0A4DF82D105E00E94CE
:1025D0006203E091D128F091D228F39708F4EDC07E
:1025E00080E09CE5A1ECB7E400E010E00093AD29A9
:1025F0001093AE2908C0EDEAF9E2008111810B5F6A
:102600001F4F008311830091AD291091AE29083628
:1026100021E012079CF52091452530914625009137
:10262000AD291091AE2975DF02E00E94620300918E
:10263000D1281091D22820E030E00E94D632AC019F
:10264000BD010E948D34B8F60091D1281091D22896
:1026500020E030E00E94D632C801D9010091AD29B6
:102660001091AE290093A9291093AA29E091D128AD
:10267000F091D228B89708F0BECF50C080E09CE51A
:10268000A1ECB7E405E010E0F4D000E010E0009326
:1026900045251093462508C0E5E4F5E20081118147
:1026A000025E1F4F0083118300914525109146253E
:1026B000083E27E0120794F52091452530914625E4
:1026C0000091A9291091AA2924DF02E00E94620347
:1026D0000091D1281091D22820E030E00E94D6321B
:1026E000AC01BD010E948D34B8F60091D128109143
:1026F000D22820E030E00E94D632C801D9010091F2
:102700004525109146250093AB291093AC29E09103
:10271000D128F091D228749708F0BECFE091A92972
:10272000F091AA29349744F0E9EAF9E20081118195
:102730000350104000831183E091AB29F091AC2944
:102740003B9744F0EBEAF9E2008111810A50104016
:10275000008311832091AB293091AC290091A929E4
:102760001091AA29D6DE0091AB291091AC290093D3
:102770006E2910936F290091A9291091AA2900931D
:102780006C2910936D2930916D29232F0EE010E0F4
:102790000E949B0A20916C290FE010E00E949B0A86
:1027A00030916F29232F00E110E00E949B0A2091B5
:1027B0006E2901E110E00E949B0A0FEF009373293C
:1027C000E4E00C9418359A938A93C80100919B29F0
:1027D000002351F020939A29409195290DE00E9401
:1027E000B2310093992907C000918D29029F009270
:1027F0006A0910926B09809366099093670904E057
:102800000093400989919991089530918D29329FC3
:1028100000926A0910926B09009366091093670988
:1028200004E00093400908950E940735D80188E02C
:1028300090E018C040918D2950E08C010E94D03169
:1028400000936A0910936B09A0936609B093670916
:1028500004E00093400908EE1DEF06DD08EB18E8E0
:1028600003DD0197813000E0900724F7E4E00C9449
:10287000183520918D2930E0220F331F20936A09EB
:1028800030936B0944E650E00E94D0310093660912
:102890001093670904E00093400948E750E0009175
:1028A000C3281091C4280E9402320E5F0E94620366
:1028B00000E00093400908958A93812F10E0D9DF4A
:1028C00000E315E7D1DC082F10E0D3DF89910895EC
:1028D00021E631E20FE915E20E94543900E80E9436
:1028E000F10200E310E0C5DF08950E94163140E0D8
:1028F00050E064E672E40E948B330E94D83208955F
:102900000E940335C801D9012A013B010091972992
:10291000002379F4A201B3018C019D010E941631BC
:1029200040E050E064E672E40E948B330E94D832AB
:1029300027C0A201B3012A013B010AE010E0209167
:10294000972930E0021B130B212F220F220B322F6D
:102950000E94CB32A801B901820193010E94043484
:10296000AC01BD010E942A33A201B3010E941631BD
:1029700040E050E064E672E40E948B330E94D8325B
:102980000B3520E0120714F00BE510E0063A2FEFAC
:10299000120714F405EA1FEFE8E00C9414350E94C6
:1029A0000335D80122E731E20FE915E20E945439DC
:1029B00000E80E94F102A13000E0B00714F180E0CD
:1029C000082F10E020E030E00E94D63228013901C3
:1029D0008D01212F220F220B322F0E94CB320E9419
:1029E0002135A801B901820193010E948D3478F547
:1029F000082F07570E9451020EE30E94950283950B
:102A0000DFCF80E008C006E8081B0E9451020CE3FB
:102A10000E9495028395082F10E020E030E00E948C
:102A2000D632280139010FEF1FEFAD010E94D031DE
:102A3000212F220F220B322F0E94CB320E942135F0
:102A4000A801B901820193010E948D34E0F200E3F4
:102A500015E70ADCE8E00C9414350E940735A0E085
:102A6000B0E000E00093010204E00E94620380E015
:102A700090E019C0E0E0F2E000810860008300917E
:102A80002B020023E1F301E000932B0200911202DC
:102A900010911302A00FB11F0091A1291091A2293A
:102AA000A01BB10B0196803A00E090071CF300E1F7
:102AB0000093010200E117E2D7DBBB2312F4A0E090
:102AC000B0E049E650E08D010E940232E4E00C944F
:102AD00018350E94073580E090E000E00093010285
:102AE00003E00E946203A0E0B0E013C0E0E0F2E087
:102AF00000810860008300912B020023E1F301E0D4
:102B000000932B020091120210911302800F911F6B
:102B10001196A43600E0B0074CF300E100930102E7
:102B200044E650E08C010E940232E4E00C94183537
:102B3000E0E0F2E0008100610083009133020023B5
:102B4000E1F301E0009333024091882950E00091C5
:102B50001402109115020E94EA310895009168292B
:102B60001091692901DC009168291091692933DCF1
:102B7000009168291091692900936A2910936B29A3
:102B800000916A2910916B29B8DB0895009168299A
:102B900010916929E9DB00916829109169291BDCF2
:102BA00000916A2910916B29A8DB4091932950E08C
:102BB0000FEF10E00E94D03145DC0091C328109146
:102BC000C428009326091093270908959A938A939D
:102BD00001E010E00E94510A902F80E002E010E036
:102BE0000E94510A10E0802B912B8093C328909370
:102BF000C42805E010E00E94510A902F80E006E012
:102C000010E00E94510A10E0802B912B80936829DC
:102C10009093692907E010E00E94510A902F80E00C
:102C200008E010E00E94510A10E0802B912B809365
:102C30006A2990936B290EE010E00E94510A902FB0
:102C400080E00FE010E00E94510A10E0802B912BF1
:102C500080936C2990936D2900E110E00E94510A45
:102C6000902F80E001E110E00E94510A10E0802BDB
:102C7000912B80936E2990936F2903E010E00E94BE
:102C8000510A0093842904E010E00E94510A009345
:102C9000852909EF11E00E94510A0093872907EF67
:102CA00011E00E94510A009390290CE010E00E946C
:102CB000510A009393290DE010E00E94510A0093FD
:102CC0008F290BEF11E00E94510A009398290CEF15
:102CD00011E00E94510A0093882906EF11E00E943A
:102CE000510A00938D2905EF11E00E94510A0093CB
:102CF00094290DEF11E00E94510A00938E2902E100
:102D000010E00E94510A009392290AE010E00E940C
:102D1000510A802F90E00BE010E00E94510A102F22
:102D200000E0802B912B80939D2990939E2903E1B5
:102D300010E00E94510A0093952908EF11E00E94CB
:102D4000510A009379290EEF11E00E94510A009375
:102D5000822904E110E00E94510A0093832900E0D7
:102D600010E00E94510A0093962904EF11E00E949E
:102D7000510A00937B2903EF11E00E94510A00934E
:102D8000972902EF11E00E94510A00939B29EDE977
:102D9000F9E20081016000838991999108950E9470
:102DA0000735D801AB3500E0B00714F0AAE5B0E074
:102DB000BB2312F48CE309C04AE050E08D010E946D
:102DC0000232102F06E0109F802D00E80E94510271
:102DD00090E0FC01E451FD4F04910E94950201E84E
:102DE0000E94510290E0FC01E351FD4F04910E94CA
:102DF000950202E80E94510290E0FC01E251FD4F71
:102E000004910E94950200EC0E94510290E0FC01A6
:102E1000E151FD4F04910E94950201EC0E94510284
:102E200090E0FC01E051FD4F04910E94950202ECFC
:102E30000E94510290E0FC01EF50FD4F04910E946E
:102E40009502BB2312F482E408C04AE050E08D01F1
:102E50000E94023206E0409F802D04E80E94510249
:102E600090E0FC01E451FD4F04910E94950205E8B9
:102E70000E94510290E0FC01E351FD4F04910E9439
:102E8000950206E80E94510290E0FC01E251FD4FDC
:102E900004910E94950204EC0E94510290E0FC0112
:102EA000E151FD4F04910E94950205EC0E945102F0
:102EB00090E0FC01E051FD4F04910E94950206EC68
:102EC0000E94510290E0FC01EF50FD4F04910E94DE
:102ED000950203E80E94510200E20E94950203EC71
:102EE0000E94510200E20E949502E4E00C94183521
:102EF0000E940735EDE9F9E2018107FF02C005E50F
:102F000001C008E53091C82833230AF47BC0209122
:102F1000C7283091C82810E0201731070CF072C084
:102F20004AE050E00091C7281091C8280E94023260
:102F3000402F4A5F00919D2910919E290E94E43103
:102F40000170002309F05EC000919029013031F436
:102F50002091782900E717E136DCACC00091902978
:102F6000023001F5E091C728F091C828759734F434
:102F70002091782900EE1EE226DC9CC00091C72833
:102F80001091C8280B3420E0120734F020917829E2
:102F900000EA1FE018DC8EC02091782900E717E1D5
:102FA00012DC88C0009190290330B9F4209178296F
:102FB000A22F8AE090E04AE050E00091C7281091EB
:102FC000C8280E940232801B910B00E416E0AC017D
:102FD0000E94D0312A2FF7DB6DC000919029043078
:102FE00009F068C02091782904E610E04091C728D4
:102FF0005091C828041B150B46E950E00E94D031BF
:10300000E2DB58C01091C82811230AF053C0009188
:10301000852910E020E030E00E94D632C801D901B5
:1030200003E010E04091C1285091C2280E94D031A5
:10303000212F220F220B322F0E94CB320E942135EA
:10304000A801B9018C019D010E948D3498F584E09E
:103050004CEE5FEF0091C7281091C8280E94023201
:10306000801B482F00919D2910919E290E94E431D8
:1030700001700023F9F40091C7281091C82800932B
:10308000CB281093CC2800917829009378290091BF
:10309000C7281091C828073E2FEF120734F020915F
:1030A000782900E21EE48FDB05C02091782900E634
:1030B0001DE689DBE4E00C9418359A938A9380919D
:1030C000C3289091C4280196AC01652F660F660B4A
:1030D000762F00E01CE62CED32E00E94693243E0DE
:1030E0000E943E3248E050E060E070E00E941632FC
:1030F00040E750E060E070E00E9469320093D7281A
:103100001093D82845E00091D7281091D8280E9424
:10311000DE3140E250E00E94D0310093D728109376
:10312000D8280091D7281091D828000F012F001F10
:1031300010E0111F0093D9281093DA2800919529E7
:103140000130A9F40091D7281091D8280093D528F0
:103150001093D62844E150E00091C3281091C42870
:103160000E9402320093DB281093DC2816C00091E5
:10317000D7281091D828000F111F0093D52810933D
:10318000D6284EE050E00091C3281091C4280E9438
:1031900002320093DB281093DC2800917F29002362
:1031A00021F400919529033041F400917F290023F7
:1031B00059F000919529033039F401E010E00093B3
:1031C000DD281093DE2806C000E010E00093DD2823
:1031D0001093DE288991999108958A93009182290C
:1031E00010E0F801E65CFC4F0491002359F10091D6
:1031F0007D29002339F59CDC2091822930E0F901FA
:10320000E65CFC4F249130E002171307DCF480E009
:1032100017C023E831E20FE915E20E94543900E8B3
:103220000E94F10208E710E024DB08EE1DEF0E9487
:10323000341101E00E94510202E00E946203839572
:10324000853038F38991089510912002137E1093F0
:1032500020020A95000F000F10912002102B1093EE
:1032600020020895B3DC29DF0E941F0200919429F7
:10327000023039F400917D29002319F40E9469116C
:1032800002C00E94451120916E2930916F29009152
:103290006C2910916D293DD979DC00919229D4DFF8
:1032A00008952091682930916929201B310B2A55F6
:1032B000304020936A2930936B2910916B29112398
:1032C00042F4EAE6F9E20081118108591E4F0083B9
:1032D00011835CDC30916B29232F07E010E00E9402
:1032E0009B0A20916A2908E010E00E949B0A089539
:1032F0000E94FB342197F89400E30E94F602E0E874
:10330000F6E0008108600083009160060F60009382
:103310006006E0E6F6E0008100620083009140066E
:103320000E6C0093400600916006006C00936006EE
:1033300008E10093110608E10093120608E10093EA
:10334000130608E10093300608E10093520608E1F5
:10335000009353060E941F020AEF11E00E94510AD7
:103360000F3F11F401E001C000E0E8E0F6E0108159
:1033700011FD0CC0E8E0F6E0108112FD07C0E8E2A4
:10338000F6E02081217011E0212701C020E0022B0E
:10339000002309F4DEC024E931E20FE915E20E94BE
:1033A000543900EC0E94F102789402E30E94620317
:1033B000F89400E00093A82905C00091A82903957E
:1033C0000093A8290091A829043008F0BDC000E0AE
:1033D0000093A72913C0B0E0FD01E759FC4F2491E9
:1033E0000A2F10E000541E4F0E949B0AA395A9309B
:1033F00090F30091A72903950093A7290091A7298D
:103400000330D8F622E001E010E00E949B0A27E595
:1034100002E010E00E949B0A20E005E010E00E941C
:103420009B0A24EB06E010E00E949B0A20E007E0E4
:1034300010E00E949B0A20EB08E010E00E949B0A2B
:1034400020E00EE010E00E949B0A20E00FE010E078
:103450000E949B0A20E000E110E00E949B0A20E00D
:1034600001E110E00E949B0A22E003E010E00E94CC
:103470009B0A22E004E010E00E949B0A20E009EF92
:1034800011E00E949B0A27E00CE010E00E949B0ADA
:1034900021E00DE010E00E949B0A21E007EF11E01F
:1034A0000E949B0A21E00AE010E00E949B0A20E8AB
:1034B0000BE010E00E949B0A20E00BEF11E00E945D
:1034C0009B0A28E10CEF11E00E949B0A27E006EF1F
:1034D00011E00E949B0A26E00DEF11E00E949B0A7A
:1034E00022E002E110E00E949B0A21E005EF11E0DA
:1034F0000E949B0A21E003E110E00E949B0A20E069
:1035000008EF11E00E949B0A22E00EEF11E00E94FA
:103510009B0A24E004E110E00E949B0A21E000E005
:1035200010E00E949B0A20E004EF11E00E949B0A39
:1035300020E003EF11E00E949B0A21E002EF11E07E
:103540000E949B0AA0E053CF20E00AEF11E00E9406
:103550009B0A0AEF11E00E94510A0093A82900E09B
:103560000093A7297FDE00919B29033018F001E02A
:1035700000939B2920919B2902EF11E00E949B0A56
:1035800003E00093852902E00093842903E200937D
:10359000010807E00093000806E910E00093260800
:1035A0001093270880918E2990E0019680932A0835
:1035B00090932B0800918E29002331F400E010E055
:1035C000009326081093270801E00093000900915A
:1035D000C3281091C428009326091093270903E0FB
:1035E000009306090091A20007600093A20007E083
:1035F0000093400804ED11E00093660810936708FB
:1036000001E0009346080E94480320916E29309102
:103610006F2900916C2910916D290E9489120E94D6
:103620001F0302E0009322020E9441030E943A031A
:103630000E941F030091922907DEA8DA02E00E948F
:10364000620347DA0093A1291093A22903E20093B1
:103650004109009164060F730093640626EA31E283
:103660000FE915E20E94543900EC0E94F10200E2D9
:1036700010E01A930A9327EB31E20FE915E20E945A
:103680005439229600E80E94F10200ED17E00E94F2
:10369000141400EA1FE00E94141400E41FE10E94C9
:1036A000141408EE1DEF0E94341100ED17E00E9483
:1036B000141400E0009340090091DB28102F06E06D
:1036C000109F002D0E94620300E61AEE0E94341142
:1036D00000919F250B3409F0B9CF0091A02500354A
:1036E00009F0B4CF0091A1250F3409F0AFCF0091BC
:1036F0008729002331F0009164060F73009364065C
:1037000005C000916406006C009364060091A22538
:10371000043509F09BCF8091A82990E001969A93F7
:103720008A932BEC31E20FE915E20E94543922967C
:1037300000EC0E94F10207EC0E945102A0E009C0D7
:103740000A2F10E000541E4F0E94510A0E94950259
:10375000A395A930A8F30091DB28102F05E0109F56
:10376000002D0E94620378940CE00E94510202E056
:103770000E94620332DDE8E0F6E0008101FD24C032
:10378000E8E0F6E0008102FD1FC00FEF00937D2905
:1037900001E000937C2901E000937E2901E00E9472
:1037A000510210E500E30E945C1424ED31E20FE9C0
:1037B00015E20E94543900E80E94F102E8E0F6E0C8
:1037C000008102FFFBCF6EC1E8E0F6E0008102FD60
:1037D00021C00FEF00937D2906E000937C2902E0D1
:1037E00000937E2901E00E94510210E500E30E944F
:1037F0005C1425EE31E20FE915E20E94543900E82D
:103800000E94F102E8E0F6E0008102FFFBCF0E9497
:10381000451148C100E000937E2900E61AEE0E949F
:1038200034111BD93801A091DB2860C04091C32816
:103830005091C4284F5F5F4F652F660F660B762F40
:1038400000E01CE62CED32E00E94693243E00E9469
:103850003E32C8017A926A929A938A9320E232E2C7
:103860000FE915E20E945439249600E80E94F10203
:103870000091D1281091D2281A930A932FE232E2B4
:103880000FE915E20E945439229600EC0E94F102E1
:103890000091952910E0000F111FF801E35BFC4F28
:1038A000059114911A930A930091962910E01A93A6
:1038B0000A930091922910E0F801E15CFC4F049119
:1038C00010E01A930A932BE332E20FE915E20E940B
:1038D0005439269609EC0E94F1020FEC0E94510225
:1038E0000AE20E94950203E00E9462030A2FA02FC1
:1038F000AA95002309F055C001E00E94510200E2A0
:103900001EE40E94341105E0601600E070060CF021
:1039100088C025E432E20FE915E20E94543900E83C
:103920000E94F10200ED10E00E94391400EB10E05B
:103930000E94391400ED10E00E94391404E10E9445
:103940006203B0C081E090E00091962910E01A93E4
:103950000A930091922910E0F801E15CFC4F049178
:1039600010E01A930A930091682910916929209117
:103970006A2930916B29021B130B1A930A939A93AD
:103980008A93B0E0BA93AA9329E032E20FE915E2F4
:103990000E9454392A9600EC0E94F10208E00E942D
:1039A0006203E8E2F6E0008100FD40CF0AE00E94F9
:1039B00062038090D1289090D2280091912910E044
:1039C0001A930A937A926A929A928A9226EF31E235
:1039D0000FE915E20E945439269600E80E94F10290
:1039E00000919D2910919E29013020E8120761F075
:1039F00000E020919D2930919E29213010E031076F
:103A000019F00060002311F0A0E001C0A1E00091D6
:103A10006E2910916F29012B09F094CF80E090E07E
:103A200093CF0091D1281091D228093522E01207B6
:103A3000C8F10091D1281091D2281A930A9323E556
:103A400032E20FE915E20E945439229603E80E94FF
:103A5000F1022DE532E20FE915E20E94543900EC43
:103A60000E94F10200ED10E00E94391400EB10E01A
:103A70000E94391400ED10E00E943914A1E010C03A
:103A800008EE1DEF0E943411E8E0F6E0008102FD2F
:103A900006C00E94DE1210E200E30E945C14A395AF
:103AA000A23370F300E00093892902E30093812997
:103AB0000093802900E010E020E030E0E3E2F9E24A
:103AC0000083118322833383E7E1F9E200831183CA
:103AD000228333830093CB281093CC280093C928EA
:103AE0001093CA28212F220F220B322FEBEFF8E27E
:103AF000008311832283338301E010E000939F2928
:103B00001093A02904E00E94620300E310E00E94E9
:103B1000391401E00093742903E00E94620300E37A
:103B200010E00E94391420C000916406006C0093DC
:103B3000640600E20093672901E0E00E00E0F01E59
:103B40008701780101342FE1120774F0EE24FF247D
:103B500044DB0091D1281091D228083E23E01207BF
:103B600018F401E00093742900917D29002309F0E5
:103B700065C40091DD281091DE28013020E0120795
:103B800009F0D1C1EBEEF8E200811181228133818D
:103B9000EFE0F9E20083118322833383EFEEF8E252
:103BA0000081118122813381EBE1F9E200831183ED
:103BB00022833383EBEFF8E2008111810093C12867
:103BC0001093C22842E050E060E070E0E7E5F9E2DF
:103BD00000811181228133810E9469320093702912
:103BE00010937129009184290D5F10918F29011B79
:103BF000009386290091862910E02091C1283091F8
:103C0000C228021713070CF02DC100917C29002354
:103C100009F028C100E000938029009181290395D3
:103C20000093812900918129003118F001E000936F
:103C30007429E3E1F9E20081118122813381EFE00F
:103C4000F9E24081518162817381401B510B620B0B
:103C5000730B4083518362837383EFE1F9E2008148
:103C6000118122813381EBE1F9E24081518162814E
:103C70007381401B510B620B730B40835183628332
:103C80007383EFE0F9E20081118122813381EFE05B
:103C9000F9E240815181628173810E941632C8012C
:103CA000D901EBE1F9E20081118122813381EBE15D
:103CB000F9E240815181628173810E941632A8012C
:103CC000B9018C019D01040F151F261F371F0E948B
:103CD000CB320E946F390E94D83228015594479404
:103CE0005594479455204AF428E004EF1EE70E94BB
:103CF000E31300E21EE40E943411EBE1F9E20081DB
:103D00001181228133810E94CB32A801B901CA01FD
:103D1000DB01EFE0F9E200811181228133810E9411
:103D2000CB32AC01BD010E9480140093C7281093D0
:103D3000C82800918129043048F1E091C728F0910A
:103D4000C828B9971CF1E091C128F091C2283A9790
:103D5000ECF0E7EFF8E200811181228133810E94CB
:103D6000CB32A801B901CA01DB01E3EFF8E200811F
:103D70001181228133810E94CB32AC01BD010E94AE
:103D800075140093C5281093C62806C000E010E003
:103D90000093C5281093C6280091C1281091C2280D
:103DA0000F5F1F4F212F220F220B322F0E94CB3289
:103DB0000E9421350E94D8320093782900917929F8
:103DC000002321F408E00093782917C00091792995
:103DD000013041F40091782910917829100F109347
:103DE00078290BC000917929023039F400917829A3
:103DF00010917829019F009278290091782910E08C
:103E000049E050E020918D2930E0421B530B0E9485
:103E100002320395009378290091C1281091C2289D
:103E2000C016D10684F40091C7281091C8280093C9
:103E3000CD281093CE2840929F295092A029C0905F
:103E4000C128D090C2280091CD281091CE2800938F
:103E5000CB281093CC280093C7281093C8280E9421
:103E60007817ECC200919B29002331F400E010E0A8
:103E700000936A0910936B09EFE0F9E20081118168
:103E800022813381E3E1F9E20083118322833383CA
:103E9000EBE1F9E20081118122813381EFE1F9E266
:103EA0000083118322833383CC24DD240091802975
:103EB00003950093802900E00093812900919B29BC
:103EC000023009F0BBC22091842930E000918F2993
:103ED00010E0200F311F00917029109171292017D7
:103EE000310794F400919929002371F400919C29E1
:103EF000039500939C29043008F4A0C222E000E559
:103F000016E40E9405149AC200E000939C290091D7
:103F10009929002309F092C200E010E000936A0999
:103F200010936B098BC200917F29002309F01BC1FC
:103F300000919529033009F016C1EBEEF8E20081FB
:103F4000118122813381E7E1F9E24081518162816F
:103F50007381041B150B260B370BEFE0F9E200838E
:103F6000118322833383EFEEF8E2008111812281F5
:103F70003381E3E2F9E24081518162817381041B64
:103F8000150B260B370BEBE1F9E20083118322833B
:103F90003383EBEFF8E2008111810093C128109385
:103FA000C228EFEEF8E200811181228133810E9464
:103FB000CB32A801B901CA01DB01EBEEF8E20081C6
:103FC0001181228133810E94CB32AC01BD010E945C
:103FD00080140093C7281093C8280091C728109117
:103FE000C828053A2FEF120761F000E02091C7289A
:103FF0003091C8282B3510E0310719F000600023FC
:1040000041F00091CB281091CC280093C728109341
:10401000C828EFE0F9E20081118122813381EFE0CD
:10402000F9E240815181628173810E941632C80198
:10403000D901EBE1F9E20081118122813381EBE1C9
:10404000F9E240815181628173810E941632A80198
:10405000B9018C019D01040F151F261F371F0E94F7
:10406000CB320E946F390E94D83245E00E94E43181
:10407000280155204AF427E000E01DE70E94E313E1
:1040800000E41CE90E943411088103950883003183
:1040900028F001E00093742900E008830091792959
:1040A000002321F408E00093782907C000917829C3
:1040B00010917829100F109378290091782910E039
:1040C00049E050E020918D2930E0421B530B0E94C3
:1040D0000232039500937829042D052939F442E032
:1040E000009178290E94B2310093782904E000936E
:1040F000400900918D29069510917829019F009221
:104100006A0910926B09E091C128F091C228319799
:10411000ECF0E091C728F091C82831976CF000E4EA
:104120001FE12091C1283091C228021B130B00937C
:104130006609109367090AC00091C1281091C2282E
:10414000005C104E009366091093670940929F2906
:104150005092A0290091C7281091C8280093CB281D
:104160001093CC286BC142E050E060E070E0EBEED1
:10417000F8E200811181228133810E946932EFE0EF
:10418000F9E2008311832283338342E050E060E050
:1041900070E0EFEEF8E200811181228133810E940C
:1041A0006932EBE1F9E2008311832283338342E039
:1041B00050E060E070E0EBEFF8E2008111812281D5
:1041C00033810E9469320093C1281093C228EFE026
:1041D000F9E20081118122813381EFE0F9E240812F
:1041E0005181628173810E941632C801D901EBE1CD
:1041F000F9E20081118122813381EBE1F9E2408112
:104200005181628173810E941632A801B9018C012B
:104210009D01040F151F261F371F0E94CB320E94DD
:104220006F390E94D83243E00E94E43128010091A6
:10423000842910E02091C1283091C2280217130769
:104240000CF0D7C000917C29002309F0D2C000E017
:104250000093802900918129039500938129E3E14E
:10426000F9E20081118122813381EFE0F9E240819E
:10427000518162817381401B510B620B730B408330
:10428000518362837383EFE1F9E20081118122811E
:104290003381EBE1F9E24081518162817381401BFE
:1042A000510B620B730B4083518362837383EBE189
:1042B000F9E200811181228133810E94CB32A80171
:1042C000B901CA01DB01EFE0F9E20081118122812D
:1042D00033810E94CB32AC01BD010E948014009357
:1042E000C7281093C82855204AF427E000E01DE7AE
:1042F0000E94E31300E41CE90E9434110091C128DC
:104300001091C2280F5F1F4F212F220F220B322F37
:104310000E94CB320E9421350E94D8320093782926
:1043200000917929002321F408E00093782917C02F
:1043300000917929013041F4009178291091782970
:10434000100F109378290BC000917929023039F4AD
:104350000091782910917829019F00927829009185
:10436000782910E049E050E020918D2930E0421B8F
:10437000530B0E9402320395009378290091812902
:10438000043098F020917829A22F80EE9EE242E03E
:1043900050E00091C1281091C2280E940232801B77
:1043A000910B8C012A2F0E94E3130091C1281091D8
:1043B000C228C016D10684F40091C7281091C828DD
:1043C0000093CD281093CE2840929F295092A02987
:1043D000C090C128D090C2280091CD281091CE283D
:1043E0000093CB281093CC280093C7281093C8289B
:1043F00025C000E000934009EFE0F9E2008111815F
:1044000022813381E3E1F9E2008311832283338344
:10441000EBE1F9E20081118122813381EFE1F9E2E0
:104420000083118322833383CC24DD2400E00093B6
:10443000812900918029039500938029009180298A
:10444000003F41F010E000918129003F19F0106019
:104450001123A9F000E010E000939F291093A029F8
:104460000093CB281093CC280093C9281093CA2816
:104470000093C5281093C62801E000937429009189
:104480007C29E2E7F3E00C94B6348091CB2890913C
:10449000CC28E0919F29F091A02934972CF08093AB
:1044A000C9289093CA2804C08091C9289091CA282D
:1044B00000919429023009F093C08C010E94CF161C
:1044C00004E610E00E94341100919F291091A02968
:1044D000212F220F220B322F0E94CB320E94213536
:1044E0000E94D832C80100918029053048F02EE69C
:1044F00032E20FE915E20E94543907EC0E94F10202
:10450000552032F403E2802E992489E090E00DC01A
:104510000091DD281091DE28012B21F40EE3802E7E
:10452000992403C006E0802E9924A0E008C00A2F39
:1045300008530E945102082D0E949502A395B0E0F5
:10454000A817B907A4F30091672910E01A930A93FA
:1045500000918F2910E01A930A930091842910E0AA
:104560001A930A930091852910E01A930A9328E779
:1045700032E20FE915E20E945439289607E80E94BA
:10458000F1020E94981548014AE050E084010E941F
:1045900002325A934A934AE050E084010E94023268
:1045A0001A930A9323E832E20FE915E20E94543984
:1045B00024960DE80E94F1020091C5281091C628AA
:1045C000013F2FEF12070CF061C507E80E9451026E
:1045D00001E20E94950200E117E20E94341156C5E3
:1045E000992352F09A938A932AE832E20FE915E26E
:1045F0000E94543922960EC04FEF5FEF8C010E944B
:10460000D0311A930A9321E932E20FE915E20E94B0
:104610005439229600E80E94F10200919F291091DE
:10462000A029212F220F220B322F0E94CB320E9471
:1046300021350E94D832C80199231AF483E290E010
:1046400006C0883000E0900711F48FEF90E004E896
:104650000E945102082F0E9495020091672910E0E4
:104660001A930A9300918F2910E01A930A930091EC
:10467000842910E01A930A930091852910E01A9377
:104680000A9328E932E20FE915E20E94543928968C
:1046900005E80E94F1020E94981548014AE050E0A6
:1046A00084010E9402325A934A934AE050E0840106
:1046B0000E9402321A930A9325EA32E20FE915E2C8
:1046C0000E94543924960DE80E94F1020091C528F9
:1046D0001091C628013F2FEF120754F406E80E94FC
:1046E000510201E20E94950200E117E20E9434119A
:1046F0000091DD281091DE28013020E0120709F03A
:104700004FC000918029063048F02BEA32E20FE9D1
:1047100015E20E94543900EC0E94F102E091C72892
:10472000F091C82831977CF00091C7281091C828D3
:10473000045C1F4F4AE050E00E9402320093CF28F1
:104740001093D02812C042E050E00091C728109189
:10475000C8280E9402320E5C1F4F4AE050E00E94BF
:1047600002320093CF281093D0280091CF28005414
:104770000E945102823000E090075CF00091802995
:10478000013020F006E00E94950203C004E00E9480
:10479000950205EC0E9451020FE20E94950276C438
:1047A00043E082010E94E431C801833C01E09007AC
:1047B00034F400E099231AF00060002311F082EC39
:1047C00091E02CEB32E20FE915E20E94543900EC43
:1047D0000E94F102A0E00FC00A2F07530E9451026D
:1047E0000EE30E94950206EC0A1B0E9451020CE3A4
:1047F0000E949502A3950A2F10E020E030E00E946D
:10480000D632480159018C01212F220F220B322F61
:104810000E94CB320E942135A801B9018401950183
:104820000E948D34C8F200ED17E00E9434112EC4AE
:104830008091A82990E001969A938A932DEC32E218
:104840000FE915E20E945439229600E80E94F10215
:1048500007E80E945102A0E009C00A2F10E00054AE
:104860001E4F0E94510A0E949502A395A930A8F3F9
:1048700000E21EE40E943411E8E2F6E0008100FD4F
:104880006CC008E210E00E9439140DE00E94510251
:10489000A0E407E0009389290FC0009189290395BE
:1048A00000938929003118F00FE000938929A0E4D2
:1048B00008E210E00E9439140091892900580E94F2
:1048C000510206E00E946203E8E0F6E0008102FF88
:1048D000E4CFE8E0F6E0008101FD10C000918929F5
:1048E0000A9500938929073018F407E00093892975
:1048F000A0E408E210E00E943914DECFE8E2F6E01E
:10490000008100FD1EC0A3950A2FA02F0B3508F0D3
:10491000A0E3AA3309F4A0E20A2F0E9495020091B5
:10492000892900580E94510202E310E00E943914C4
:104930002A2F0091892910E007541E4F0E949B0ADC
:10494000BBCFE8E0F6E0008103FDB6CF08E210E05F
:104950000E9439140CE00E9451020E94451126ED7C
:1049600032E20FE915E20E94543900EC0E94F10294
:10497000A0E010C00A2F0A530E9451020A2F0E9481
:104980009502A83031F40EEC0E9451020FEF0E9404
:104990009502A3958091A82990E00196B0E08A172E
:1049A0009B0744F773C30E949815C8014AE050E082
:1049B0008C010E9402325A934A934AE050E08C01E3
:1049C0000E9402321A930A930091822910E0F801A2
:1049D000E65CFC4F04914AE00E94B23150E05A93E9
:1049E0004A930091822910E0F801E65CFC4F0491A3
:1049F0004AE00E94B23110E01A930A9327EE32E2A5
:104A00000FE915E20E945439289600E80E94F1024D
:104A10000091882910E01A930A932DEF32E20FE9F2
:104A200015E20E945439229600EC0E94F10202E045
:104A30000E9462032BC300918E2910E01A930A93FF
:104A40002EE033E20FE915E20E945439229600E885
:104A50000E94F10220E233E20FE915E20E9454398C
:104A600000EC0E94F102A0E010C00A2F0A530E943D
:104A700051020A2F0E949502A83031F40EEC0E94D8
:104A800051020FEF0E949502A39500918E290A17FB
:104A900060F702E00E946203F9C20E942D15C8016E
:104AA0009A938A9322E333E20FE915E20E94543984
:104AB000229600E80E94F1020091D5281091D62894
:104AC0001A930A9325E433E20FE915E20E94543960
:104AD000229609E80E94F1024091C3285091C4280F
:104AE0004F5F5F4F652F660F660B762F00E01CE669
:104AF0002CED32E00E94693243E00E943E323A934C
:104B00002A931A930A932EE433E20FE915E20E94E6
:104B10005439249600EC0E94F10200E21EE40E9447
:104B20003411B4C240E250E060E070E0EFEEF8E231
:104B300000811181228133810E9469320E94CF1449
:104B40002EE533E20FE915E20E94543900EC0E9491
:104B5000F1020FED10E01A930A9300916829109169
:104B600069291A930A9329E633E20FE915E20E94B4
:104B7000543924960AEC0E94F10200E21EE40E94DD
:104B8000341184C200917B29002311F4A3E501C0F4
:104B9000ADE40E942D151A930A9322E733E20FE940
:104BA00015E20E945439229600E80E94F102B0E01A
:104BB000BA93AA932AE733E20FE915E20E94543927
:104BC000229606E80E94F10226E833E20FE915E298
:104BD0000E94543900EC0E94F102A0E010C00A2F9C
:104BE0000A530E9451020A2F0E949502A83031F404
:104BF0000EEC0E9451020FEF0E949502A3950091C6
:104C000093290A1760F702E00E9462033FC20091F5
:104C1000962910E01A930A930091922910E0F80166
:104C2000E15CFC4F049110E01A930A9327E933E208
:104C30000FE915E20E945439249600E80E94F1021F
:104C400020EA33E20FE915E20E94543906E80E9497
:104C5000F1022BEA33E20FE915E20E94543900EC2D
:104C60000E94F102A0E010C00A2F0A530E945102D4
:104C70000A2F0E949502A83031F40EEC0E945102D6
:104C80000FEF0E949502A395009192290A1760F7F1
:104C900002E00E946203FAC10091D1281091D2284B
:104CA0001A930A932CEB33E20FE915E20E94543970
:104CB000229600E80E94F10200916E2910916F295E
:104CC0001A930A9327EC33E20FE915E20E94543954
:104CD000229609E80E94F1020FED10E01A930A9360
:104CE00000916C2910916D291A930A9320ED33E2FB
:104CF0000FE915E20E945439249600EC0E94F1025B
:104D000000917329002321F409E80E94510203C095
:104D100009EC0E9451020EE30E94950202E00E94FB
:104D20006203B4C10091832910E01A930A9323EE21
:104D300033E20FE915E20E945439229600E80E94FE
:104D4000F10220EA33E20FE915E20E94543906E845
:104D50000E94F1022BEE33E20FE915E20E94543972
:104D600000EC0E94F102A0E010C00A2F0A530E943A
:104D700051020A2F0E949502A83031F40EEC0E94D5
:104D800051020FEF0E949502A395009183290A1703
:104D900060F702E00E94620379C144E050E060E005
:104DA00070E0EBEFF8E200811181228133810E94F3
:104DB00069320E94CF142CEF33E20FE915E20E9412
:104DC000543900EC0E94F1020FED10E01A930A939F
:104DD00000916A2910916B291A930A9329E633E20C
:104DE0000FE915E20E94543924960AEC0E94F10260
:104DF00000E41CE90E94341149C10091792910E0B6
:104E0000000F111FF801EB5AFC4F059114911A93F2
:104E10000A9328E034E20FE915E20E945439229601
:104E200000E80E94F10220EA33E20FE915E20E9455
:104E3000543906E80E94F1022FE034E20FE915E24E
:104E40000E94543900EC0E94F102A0E010C00A2F29
:104E50000A530E9451020A2F0E949502A83031F491
:104E60000EEC0E9451020FEF0E949502A395009153
:104E70008D290A1760F700E61AEE0E94341106C168
:104E800000919029033019F48AE090E00CC0009161
:104E90009029043019F48AE590E005C080919029AA
:104EA00090E0880F991F9A938A9320E234E20FE9E9
:104EB00015E20E945439229600E80E94F102009106
:104EC0009B2910E0000F111FF801E55AFC4F0591D6
:104ED00014911A930A9329E234E20FE915E20E9431
:104EE0005439229607E80E94F10222E334E20FE9E6
:104EF00015E20E94543900EC0E94F102A0E008C0C3
:104F00000A2F06530E9451020A2F0E949502A39570
:104F1000009190290A17A0F702E00E946203B6C030
:104F20000091972910E01A930A930091942910E0B8
:104F3000000F111FF801E15AFC4F059114911A93CB
:104F40000A9323E434E20FE915E20E9454392496CF
:104F500000E80E94F10223E534E20FE915E20E9425
:104F6000543900EC0E94F102A0E010C00A2F0A534D
:104F70000E9451020A2F0E949502A83031F40EECD3
:104F80000E9451020FEF0E949502A395009197296C
:104F90000A1760F702E00E94620378C00091952929
:104FA00010E0000F111FF801E35BFC4F0591149115
:104FB0001A930A9324E634E20FE915E20E94543969
:104FC000229600E80E94F10222E734E20FE915E29E
:104FD0000E94543900EC0E94F102A0E010C00A2F98
:104FE0000A530E9451020A2F0E949502A83031F400
:104FF0000EEC0E9451020FEF0E949502A3950091C2
:1050000095290A1760F702E00E94620301E000930D
:1050100076293CC0009176290023C1F124E834E2CE
:105020000FE915E20E94543900E80E94F102A0E065
:1050300004C000E20E949502A395A03190F40A2FCB
:1050400000540E9451024A2F00919D2910919E29DF
:105050000E94E4310170002361F303E20E94950293
:10506000EBCF05EC0E9451020FE20E9495020091E5
:10507000892900540E9451020EE00E94510200E072
:105080000093762908EE1DEF0E943411B0E0E8E0AD
:10509000F6E0008103FDC7C000E00093400901E095
:1050A0000093742900917A290130B1F406E210E0EE
:1050B0000E943914E8E0F6E0008103FFFBCF01E035
:1050C0000093742904EB009381290093802900E068
:1050D00000937A290C940331E8E0F6E0008103FDA7
:1050E00054C008EE1DEF0E943411B3950B2FB02F62
:1050F0002091DB283091DC2810E02017310760F781
:1051000000917D29009500937D2901E000937A2983
:1051100000919429023019F40E94691102C00E9482
:10512000451101E00E94510200917D29002381F484
:1051300000E000937C294091932950E00FEF10E0AC
:105140000E94D0310E94221202E00E9462030CC031
:105150000BE000937C2902E00E94620300E010E073
:105160000E9422120E94451101E00093762900E07E
:1051700000937E2900E000937F290AE510E00E9459
:10518000391401E000937429A9C100917D290023FD
:1051900069F400917F29009500937F290E945D1892
:1051A00004EB009381290093802938C00CE00E9411
:1051B000510200917E29013059F400917C29039518
:1051C00000937C290B30E8F001E000937C2919C0A2
:1051D00000917E29023059F400917C2903950093B7
:1051E0007C290B3070F006E000937C290AC0009106
:1051F0007C29039500937C29003118F001E000938D
:105200007C2900917C290C3049F44091932950E08D
:105210000FEF10E00E94D0310E94221208E210E04D
:105220000E943914EDC7E8E2F6E0008100FDB6C344
:1052300000E00093400900917C29E8E9F3E00C9438
:10524000B63401E00E94510200E21EE40E943411D3
:10525000E8E2F6E0008100FD0FC008EE1DEF0E94BD
:105260003411B3950B2FB02F2091DB283091DC281F
:1052700010E02017310760F7B3950B2FB02F209166
:10528000DB283091DC2810E02017310708F072C0CD
:10529000E7EFF8E200811181228133810E94CB3255
:1052A000A801B901CA01DB01E3EFF8E20081118135
:1052B000228133810E94CB32AC01BD010E94801457
:1052C0000093C7281093C828E3EFF8E2008111810A
:1052D00022813381E7E1F9E2008311832283338362
:1052E000E7EFF8E20081118122813381E3E2F9E204
:1052F00000831183228333830091C7281091C8282B
:105300000F3C2FEF120764F400E02091C728309182
:10531000C828263A1FEF31071CF00060002391F0E7
:1053200025E934E20FE915E20E94543900EC0E94AD
:10533000F10200EA10E00E94391400EB10E00E9434
:1053400039146CC026EA34E20FE915E20E945439A0
:1053500000EC0E94F1020091C7281091C8280E9419
:10536000511900E510E00E94391400E210E00E949B
:10537000391454C001E0009374290091D128109190
:10538000D2281A930A9327EB34E20FE915E20E9420
:105390005439229600E80E94F10200E310E00E94D6
:1053A000391400918129002311F401E001C000E0CB
:1053B0000093802908E00E94620322C78201212F06
:1053C000220F220B322F0E94CB320E9421354091B6
:1053D000C7285091C8285A934A9340E050E060E0B3
:1053E00070E40E948B330E94D8321A930A9329ECFE
:1053F00034E20FE915E20E945439249600E80E9435
:10540000F10222E000E41FE1E7E5F9E24081518189
:10541000440F551F041B150B0E94E313E8E2F6E04E
:10542000008100FD4CC0E8E0F6E0008102FD15C0FF
:10543000E7ECF8E2008111810F5F1F4F00831183B9
:105440000091C7281091C8280E94511900E410E06B
:105450000E94391406E00E946203E8E0F6E0008151
:1054600001FD15C0E7ECF8E2008111810150104008
:10547000008311830091C7281091C8280E945119F8
:1054800000E410E00E94391406E00E946203E8E0A4
:10549000F6E0008103FD92CF00E310E00E94391492
:1054A00026EA34E20FE915E20E94543900EC0E942A
:1054B000F1020091C7281091C8280E94511900E0FC
:1054C000009340090AE00E9462032EED34E20FE9E6
:1054D00015E20E94543900EC0E94F10291C600913D
:1054E0008229039500938229053018F000E000938B
:1054F0008229209182290EEF11E00E949B0A0091DF
:10550000DB281091DC280E94341102E310E00E9495
:10551000391476C6A0E0B0E00E9468148DE591E0F1
:1055200012C0809326099093270904E00E94620329
:105530000E942D15A017B1072CF4D8018093C32821
:105540009093C4280496873E03E0900754F300919B
:10555000C3281091C42800932609109327090E949C
:105560005D1810E400E50E945C143091C428232FDC
:1055700001E010E00E949B0A2091C32802E010E0A5
:105580000E949B0A3DC621E135E20FE915E20E9427
:10559000543900E80E94F10200E810E00E9439143A
:1055A00000E810E00E943914E8E2F6E0008100FD16
:1055B000E9C000E61AEE0E943411B3950B2FB02F0C
:1055C0002091DB283091DC2810E02017310760F7AC
:1055D00001E0009377292FEE34E20FE915E20E94F3
:1055E000543900E80E94F10200E310E00E943914EF
:1055F00001E00093742902E30E94620320E035E297
:105600000FE915E20E94543900E80E94F10200E31C
:1056100010E00E94391408E20E94620380E090E0EA
:10562000A0E01EC0E7EFF8E2008111812281338102
:105630000E94CB32A801B9014A015B01E3EFF8E215
:1056400000811181228133810E94CB32A401B501F6
:105650000E947514800F911F08E00E946203A395B9
:10566000AA3000F34AE050E08C010E940232C801E7
:10567000E0916829F0916929EA55F040E81BF90B9F
:10568000E0936829F09369290091682910916929AC
:10569000093621E0120744F0E8E6F9E200811181C1
:1056A000085611400083118310916929112342F497
:1056B000E8E6F9E20081118108591E4F0083118349
:1056C0000E94AE150091DB280E946203E7EFF8E22A
:1056D00000811181228133810E94CB32A801B9015E
:1056E0004A015B01E3EFF8E20081118122813381FD
:1056F0000E94CB32A401B5010E94751448010CEA46
:1057000080160FEF90060CF03ECF22E235E20FE953
:1057100015E20E94543900E80E94F10205E210E00F
:105720000E94391405E00E94620305E210E00E9425
:105730003914009168291091692900936A291093FE
:105740006B2900916A2910916B290E947D1130917B
:105750006929232F05E010E00E949B0A2091682907
:1057600006E010E00E949B0A30916B29232F07E08E
:1057700010E00E949B0A20916A2908E010E00E9434
:105780009B0A12CF00917729002389F423E335E2A5
:105790000FE915E20E94543900E80E94F10208EE78
:1057A0001DEF0E94341100E510E00E94391428C555
:1057B00000917B29002321F401E000937B2903C0A1
:1057C00000E000937B294091932950E00FEF10E017
:1057D0000E94D0310E94221220917B2904EF11E017
:1057E0000E949B0A02E310E00E94391404E00E9428
:1057F000620306C50091962903950093962903300C
:1058000018F001E0009396292091962900E010E01D
:105810000E949B0A02E310E00E94391404E00E94F7
:105820006203EEC4E8E2F6E0008100FD1AC008EE73
:105830001DEF0E943411B3950B2FB02F2091DB2860
:105840003091DC2810E02017310760F700E610E007
:105850000E9439140E94DE1210E200E30E945C14E0
:10586000CFC40091732900950093732902E310E0DF
:105870000E94391405E00E946203C2C40091792994
:10588000039500937929033018F000E000937929FB
:105890002091792908EF11E00E949B0A02E310E0B1
:1058A0000E94341102E310E00E943914A9C400914F
:1058B0009B29039500939B29033018F000E0009387
:1058C0009B2920919B2902EF11E00E949B0A02E391
:1058D00010E00E94391408E00E94620391C4009114
:1058E0009429039500939429033018F001E0009364
:1058F00094292091942905EF11E00E949B0A02E36C
:1059000010E00E94391404E00E94620379C481E02F
:1059100090E0409189298C010E94D831C8014091C2
:10592000892900919D2910919E290E94E4310170DE
:10593000002379F080959095EDE9F9E200811181DD
:10594000082319230083118310E500E40E945C14EE
:105950000CC0EDE9F9E200811181082B192B0083BD
:10596000118310E300E40E945C1401E000937629A7
:1059700020919D290AE010E00E949B0A30919E2907
:10598000232F0BE010E00E949B0A3AC401E0009331
:10599000742908E210E00E94391432C4E8E0F6E00D
:1059A000008102FD1EC200E00093400900917C29A5
:1059B000EEEBF3E00C94B634E8E0F6E0008102FD93
:1059C00025C000E61AEE0E943411B3950B2FB02FBC
:1059D0002091DB283091DC2810E02017310760F798
:1059E000009187290095009387292091872909EF45
:1059F00011E00E949B0A01E00093772900E510E086
:105A00000E94391401E00E946203FDC300917729CE
:105A1000002381F4009184290395009384290A309E
:105A200018F000E0009384292091842903E010E01D
:105A30000E949B0ACEC10091A82903950093A82932
:105A4000043018F003E00093A8290E943219209135
:105A5000A8290AEF11E00E949B0ABBC10091882986
:105A60000395009388290D3318F001E000938829ED
:105A7000209188290CEF11E00E949B0A00E41CE9A8
:105A80000E943411A6C100918E29039500938E299E
:105A9000093018F008E000938E290BE910E000931C
:105AA00026081093270820918E290DEF11E00E94FF
:105AB0009B0A80918E2990E0019680932A0890930A
:105AC0002B0887C18091C3289091C42801978093A7
:105AD000C3289093C4288D3501E0900734F40DE578
:105AE00011E00093C3281093C4280091C32810919B
:105AF000C42800932609109327090E945D1830914D
:105B0000C428232F01E010E00E949B0A2091C328A3
:105B100002E010E00E949B0A5CC18091682990918C
:105B2000692901968093682990936929883601E054
:105B3000900734F000E010E0009368291093692981
:105B40000E94AE15009168291091692900936A2975
:105B500010936B2930916929232F05E010E00E94F2
:105B60009B0A2091682906E010E00E949B0A31C13F
:105B700000919329039500939329093018F008E0C8
:105B8000009393294091932950E00FEF10E00E9479
:105B9000D0310E942212209193290CE010E00E9443
:105BA0009B0A17C10091922903950093922908300E
:105BB00018F007E000939229009192290E9424197D
:105BC0002091922902E110E00E949B0A02C1E8E0C4
:105BD000F6E0008101FD1BC000E010E000936E299B
:105BE00010936F2900936C2910936D2904E610E03F
:105BF0000E94391406E00E94620320E00EE010E0EB
:105C00000E949B0A20E00FE010E00E949B0A009196
:105C10007329002309F580916E2990916F290196CF
:105C200080936E2990936F29813008E0900734F0BB
:105C300000E018E000936E2910936F2930916F29CE
:105C4000232F00E110E00E949B0A20916E2901E1C0
:105C500010E00E949B0A20C080916C2990916D29D0
:105C6000019680936C2990936D29883601E0900706
:105C700034F000E010E000936C2910936D2930910E
:105C80006D29232F0EE010E00E949B0A20916C29C1
:105C90000FE010E00E949B0A20916E2930916F293D
:105CA00000916C2910916D290E94891202E00E94D6
:105CB00062038FC0009183290395009383290930E3
:105CC00018F008E0009383292091832904E110E073
:105CD0000E949B0A7EC080916A2990916B2901964F
:105CE00080936A2990936B29883601E0900734F0FD
:105CF00000E010E000936A2910936B2900916A2953
:105D000010916B290E947D1130916B29232F07E0A0
:105D100010E00E949B0A20916A2908E010E00E948E
:105D20009B0A57C000918D29039500938D29093056
:105D300018F008E000938D2920918D2906EF11E0DD
:105D40000E949B0A46C000919029039500939029D8
:105D5000053018F004E0009390292091902907EF76
:105D600011E00E949B0A35C000919729039500938A
:105D70009729093018F008E0009397292091972976
:105D800003EF11E00E949B0A24C00091952903951E
:105D900000939529043018F003E0009395290091B1
:105DA00092290E9424192091952903E110E00E9474
:105DB0009B0A0E945D180DC00091892903950093EC
:105DC0008929003118F000E00093892901E000934F
:105DD000762908E210E00E94391401E0009374294A
:105DE0000FC2E8E0F6E0008101FD0AC200E0009386
:105DF000400900917C29E4EEF3E00C94B634E8E02D
:105E0000F6E0008101FD2AC000E61AEE0E9434117E
:105E1000B3950B2FB02F2091DB283091DC2810E0B8
:105E20002017310760F700918F29039500938F2980
:105E3000053018F001E000938F2920918F290DE0A3
:105E400010E00E949B0A01E00093772900E510E032
:105E50000E94391403E00E946203D5C100917729A2
:105E6000002381F4009185290395009385290A3048
:105E700018F000E0009385292091852904E010E0C6
:105E80000E949B0AB6C10091A8290A950093A829EF
:105E90000F3F19F400E00093A8290E9432192091C5
:105EA000A8290AEF11E00E949B0AA3C1009188294A
:105EB0000A9500938829002319F40CE3009388299C
:105EC000209188290CEF11E00E949B0A00E41CE954
:105ED0000E9434118EC100918E290A9500938E295B
:105EE0000F3F19F400E000938E2920918E290DEFC9
:105EF00011E00E949B0A80918E2990E00196809388
:105F00002A0890932B0875C18091C3289091C428CA
:105F100001968093C3289093C428883E03E090079D
:105F200034F007EE13E00093C3281093C4280091C7
:105F3000C3281091C42800932609109327090E94B2
:105F40005D183091C428232F01E010E00E949B0AC5
:105F50002091C32802E010E00E949B0A4AC1809170
:105F600068299091692901978093682990936929FC
:105F7000992332F408E611E0009368291093692907
:105F80000E94AE15009168291091692900936A2931
:105F900010936B2930916929232F05E010E00E94AE
:105FA0009B0A2091682906E010E00E949B0A21C10B
:105FB000009193290A95009393290F3F19F400E06B
:105FC000009393294091932950E00FEF10E00E9435
:105FD000D0310E942212209193290CE010E00E94FF
:105FE0009B0A07C1009192290A95009392290130DA
:105FF00018F401E000939229009192290E9424193B
:106000002091922902E110E00E949B0AF2C0E8E090
:10601000F6E0008102FD11C000E010E000936E295F
:1060200010936F2900936C2910936D2904E610E0FA
:106030000E94391406E00E94620300917329002334
:10604000F9F480916E2990916F29019780936E29C0
:1060500090936F29992332F400E010E000936E29A9
:1060600010936F2930916F29232F00E110E00E94D7
:106070009B0A20916E2901E110E00E949B0A1EC03C
:1060800080916C2990916D29019780936C29909350
:106090006D29992332F407E611E000936C291093DF
:1060A0006D2930916D29232F0EE010E00E949B0A8C
:1060B00020916C290FE010E00E949B0A20916E292C
:1060C00030916F2900916C2910916D290E948912DD
:1060D00002E00E9462038DC0009183290A9500931B
:1060E00083290F3F19F400E000938329209183292D
:1060F00004E110E00E949B0A7CC080916A29909183
:106100006B29019780936A2990936B29892B31F42D
:1061100008E611E000936A2910936B2900916A291F
:1061200010916B290E947D1130916B29232F07E07C
:1061300010E00E949B0A20916A2908E010E00E946A
:106140009B0A57C000918D290A9500938D290F3F16
:1061500019F400E000938D2920918D2906EF11E0BC
:106160000E949B0A46C0009190290A9500939029AD
:10617000013018F401E0009390292091902907EF55
:1061800011E00E949B0A35C0009197290A9500935F
:1061900097290F3F19F400E0009397292091972940
:1061A00003EF11E00E949B0A24C0009195290A95F3
:1061B00000939529013018F401E00093952900918E
:1061C00092290E9424192091952903E110E00E9450
:1061D0009B0A0E945D180DC0009189290A950093C1
:1061E00089290F3F19F40FE00093892901E00093FA
:1061F000762908E210E00E94391401E00093742926
:1062000000E00093772900918729002311F40C9472
:10621000941D009164060F73009364060AE20093D4
:1062200067290C949C1D00008895FECF0E940335C1
:10623000C801D9012A013B015CD057D071F4820119
:10624000930153D051F401E2EFEAF9E20083418374
:106250000FEF1FEF2FE73FE73DC044D0A201B3018E
:106260000E942A33AC01BD0140D061F442D03AD043
:106270000E94A5340BED1FE029EC10F43FE32AC087
:106280003FEB28C0A201B3012DD00E9404340801C5
:1062900019012FD0820193010E948D3423D0A0F4E4
:1062A0001CD050F424D0A801B9010BED1FE029E463
:1062B00030E40E946E330EC01AD04BED5FE069E40B
:1062C00070EC0E942A3306C008D010F410D002C02F
:1062D0000ED03058E8E00C9414350E94A5348001AB
:1062E000910108958C019D0108950C9483340C94C0
:1062F000053840E050E060E070E008953F7741E00D
:106300000C94A43803E20DBF01E20EBFC0E0D1E25D
:106310000E94A435002311F00E9487380E9478194A
:106320000E9413310C9413310D01DA0140E050E06A
:1063300060E070E00E94833439F400E010E04D9397
:106340004C9320E030E00CC0B901660F771F7E57F8
:10635000572F550F550B7D935C932F7730783F6304
:10636000D00108950024E8E0EA9532F0001F001CF7
:106370000416D0F3041AF8CF001F402D009508959D
:10638000FF27442312F4F1604195002312F4F095A5
:1063900001950E94B231F0FD0195F1FD41950895FE
:1063A000149F102D059F100D049F002D110D0895B1
:1063B0004A951AF0000F111FFBCF08954A951AF065
:1063C00016950795FBCF08954A951AF015950795F0
:1063D000FBCF089500241124EFE0001F111F001CC3
:1063E000111C0416150610F0041A150AEA95AAF7EE
:1063F000001F111FA001009510950895519541951A
:1064000050400895FF27552312F4F160F7DF112360
:1064100012F4F09507D00E94EA31F0FD03D0F1FDAF
:10642000EDCF089511950195104008952224349FD1
:10643000302D259F300D169F300D079F300D249F66
:10644000202D310D159F200D311D069F200D311D72
:10645000149F102D210D321D059F100D211D321D81
:10646000049F002D110D221D321D08954A952AF01A
:106470003695279517950795F9CF08954A952AF0EF
:106480003595279517950795F9CF08950024112480
:106490001001E0E2EA9592F0001F111F221F331F46
:1064A000001C111C221C331C041615062606370678
:1064B00088F3041A150A260A370AECCF001F111FA9
:1064C000221F331FA001B101009510952095309532
:1064D0000895FF27772312F4F16015D0332312F4C7
:1064E000F09509D00E944632F69508F404D0F6954E
:1064F00008F409C0089530952095109501951F4F17
:106500002F4F3F4F089570956095509541955F4F7F
:106510006F4F7F4F0895FF27112477FB660F771F7A
:10652000089409F4771F679517F8EE27002437FBC6
:10653000220F331F089409F4331F279507F8089595
:1065400027FD0EC0EE0F001F111F221F3A9532309B
:10655000B8F7332319F427FD31E002C027FF30E0FC
:10656000E03821F400FF08940EF488940F4F1F4F79
:106570002F4F3F4F323038F4332319F427FD31E0E9
:1065800002C027FF30E03F3F29F0220F000C379573
:1065900027950895ACC0032E002012F40E947B3290
:1065A000E02F012F122F232F3EE9D1CF0024F8CF67
:1065B000BCDF432F4F5748F04F3148F007FC91C0E4
:1065C0003FE72FEF1FEF0FEF089533278CC0322FD7
:1065D000212F102F0E2F4F5141950E94363207FE6A
:1065E00008950C947B32F901EE0FFF1F37FBFF3F3C
:1065F00031F0EF2BE12BE02B8894B8940895E02B39
:10660000E12B21F008949894B89408959894889474
:1066100038940895FB01EE0FFF1F77FBFF3F31F029
:10662000EF2BE52BE42B8894B8940895E42BE52B0D
:1066300069F3E8CFEFDF68F021F43723262F8A01D2
:106640000895372FFBCFE6DF20F00BF00895732776
:10665000EAF751C0C8DFE8F3B3F361F3DBDFC8F357
:1066600083F3A1F358DF401751076207730731F432
:10667000011411F10024E89488942BC078F0332E93
:10668000372F732D322E262F632D312E152F532D9C
:10669000302E042F432D302C012C132C371739F0BA
:1066A000669557954795F795E0407395F7CFE7FBCB
:1066B000EE0FE0E010246AF0EF0F041F151F261FF5
:1066C00060F4279517950795E79508F46894339536
:1066D0003ECFEF0B040B150B260B39CFE0E87E27DE
:1066E000B9CF302D307822271127002708953FE7B2
:1066F000302920E8F9CF3FEF2FEFF6CF8BDFD8F32B
:10670000D1F370783727089585DFA8F3A3F3F9CF85
:106710003078372793CF67DF70F383F3A9F37ADFFD
:1067200050F3B3F3A9F3F7DE0124E8943F57E040B8
:10673000370FEF1F12F0D9F603C03A3E90F268947B
:10674000E0E00A92AA933A93AA273324222433271B
:10675000049FF001059FF00D712D731F149FF00D24
:10676000711D221C069F700D211C331C159F700D7E
:10677000211C331E249F700D211C331E169F200CDC
:10678000311CAA1F259F200C311CA31F269F300CF3
:10679000A11D39915EF43395A6953794279477958A
:1067A000F795E79533953130BCF316C0AA2322F054
:1067B000332351F4339510C0339571F4A9910990A6
:1067C00096CFA7FD09C03A95EE0FFF1F771F221C39
:1067D000331CAA1F3230A8F7E894FE2B09F0689406
:1067E0002A2F8101E72FA9910990BACE13DF10F06B
:1067F0000BF087CF80CF0EDFE9F3E0F3032E0726FF
:1068000070CF032E072673CFEEDEA0F37BF399F350
:1068100001DF80F39BF3A9F37EDE012427FD06C090
:10682000000F111F221F3150E040F8CF67FD06C056
:10683000440F551F661F7150F040F8CFE894371B86
:10684000EF0B3158EF4F2AF0EE23E9F63F3FD9F234
:1068500003C03A3EA8F26894E0E0F0E011241394FB
:1068600040175107620738F0315008F46894000F60
:10687000111F221FEE1F041B150B260BEF0B000F21
:10688000111F221FEE1F0A9279E17A95AAF00417D0
:1068900015072607EF0730F0041B150B260BEF0B2F
:1068A000089401C08894111C221C331C001C000F8A
:1068B000111F221FEE1FE9CFF0F9E894E22BE12B24
:1068C000E02B09F068940694379427941794E79581
:1068D00008F468947395B9F30990332311F0F0FF2D
:1068E00009C0369427941794E79508F46894339573
:1068F0003130BCF3012D122D232D32CE8BCE989446
:106900000895189408956FDED0F3C1F383DEB8F3D1
:10691000041715072607370708957CDEA0F063DE0D
:1069200090F029F0E32FE7273AF47317089572DE09
:1069300051F04EF0089408950417150726073707FD
:1069400019F016F4B8F78894089564DEE0F34BDE8E
:10695000D0F3E7DFC0F308940895759165915591E0
:106960004591159011FA259035900895F9DF041B93
:1069700010E003C0F4DF041B150B20E030E005C07D
:10698000ECDF041B150B260B370BB8F010FC17C0FF
:1069900045910590E00FF11F0417100540E0240712
:1069A000340758F436F404910024F101E01BF00997
:1069B0000994E00FF11F25903590F101099411F42D
:1069C000D6F7F1CF31960EF0319650E060E070E0EE
:1069D00045914B3F48F089F34F3F29F04E3F11F06E
:1069E0007591659155914591041B150B260B370B3D
:1069F00039F318F3E7CFFA92EA92DA92CA92BA928E
:106A0000AA929A928A927A926A925A924A92BA93E5
:106A1000AA939A938A930895FF84EE84DD84CC84AC
:106A2000BB84AA84998488847F806E805D804C803A
:106A3000BB81AA8199818881F0E0EC0FFD1FEF01F5
:106A400008950E94FF34229741E050E060E070E03A
:106A50000E948D3460F440E00E94833421F402E20D
:106A60006BD03FEF5FC001E267D03FE75BC0AE0194
:106A70000E949431C801D90143EF54E065E37FE3FC
:106A80000E948D3468F437FBAA0FBB1FB395B695EF
:106A9000A795B7F90881198101501040088319831F
:106AA00040E050E060E87FEB43D02801390140E04E
:106AB00050E060E87FE33CD0A801B9018201930176
:106AC0000E940434C801D901A801B9012FD02801BE
:106AD00039010881102F110F110B212F312F0E9426
:106AE000CB3248E152E761E37FE320D0480159010E
:106AF00042E252E964ED7EE38201930117D04DED4D
:106B00005BE96AE27FE316D0A201B3010FD044E053
:106B100050E060E070E40ED0AC01BD0107D0A401EC
:106B2000B50108D02296ECE00C9410350C948B3310
:106B30008C019D010C942A33EFEAF9E20083518322
:106B40000FEF1FEF2FE7089501E008950E94FB3437
:106B5000EF97EF976A972A873B874887598768019D
:106B60007B0100E00B830C8302C011D21BD20AD23E
:106B7000053251F00023C9F70B811C81EF96EF9687
:106B80006A96E0E10C940C350081053221F402D2C2
:106B9000FED105E2EBCF00E00F830E830A83098369
:106BA0003E0102E1600E00E0701E07E415E2088B72
:106BB000198B06C00981002311F400810983EAD1F1
:106BC000D9D10052B9F3035059F00850B1F3025033
:106BD00019F0035049F00CC00A8103950A83EFCFE6
:106BE0000E8103950E83EBCF0F8103950F83E7CFC3
:106BF00000810A3279F4AAD1AD90BD9098D1BB2022
:106C00003AF4B194A19400E0B00A0A8103950A8392
:106C1000C1D114C0AA24BB244AE050E00DC0219188
:106C20006F0185010E94D031A22EBB24A00EB11E9F
:106C300000EDA00E0FEFB01EA0D188F30A81002353
:106C400011F000E00F8396D10E32F1F4A3D192D16E
:106C50000A3231F47BD18D909D9069D19BD117C0C0
:106C6000882499244AE050E088D188F421916F016A
:106C700084010E94D031822E9924800E911E00ED55
:106C8000800E0FEF901EF0CF88248A94982C80E01D
:106C900071D10C5421F00C5131F0045039F481E0E1
:106CA000C80E7AD103C001E0C00ED81E6BD1EAE055
:106CB000F4E00C94B63480FB5EF44B815C81652F6C
:106CC000660F660B47D140835183628363834FCF46
:106CD0002B813C813FD12083318349CF37D10D9126
:106CE000119625D10A8B2E0103E115D1E0C02ED1DA
:106CF0006D907D901CD1062D072921F408E5602EAA
:106D000005E2702E992022F400E1802E07E2902EF9
:106D100080E090E001C00196F30101913F01002362
:106D200019F088159905BCF30CD123019195819533
:106D30009040680E791EBBC00E81002331F0082DF3
:106D4000092919F499248824839407E615E2088B0D
:106D5000198B0881003739F4F9D0ECD000E1D5D097
:106D600000E0098330C0F1D046F40D911D912D91C2
:106D70003D91DDD0C801D90101C0DCD008810F36BA
:106D800011F408E0ECCF053749F70AE0E8CFDDD091
:106D90004D915D9126F46D917D91C9D005C0C7D00C
:106DA000652F660F660B762FCA01DB0177234AF445
:106DB0000DE209839095A095B09581959F4FAF4FB7
:106DC000BF4F0AE0A2D03E0107E9600E00E0701E4E
:106DD0002E0107E9A0D0082F092B0A2B0B2B11F04D
:106DE00001E001C000E00D83082D092919F40D818F
:106DF00000FF1FC094D0E889F989E00DF11D0081E2
:106E0000F30102933F018BD0C801D901012B022B62
:106E1000032B81F799206AF40F81002351F0A3D04E
:106E200010E04501801A910A04C000E3F3010293C7
:106E30003F018E0109561F4F06191709081519053C
:106E4000A4F30E81002399F10D8100FF30C0088169
:106E5000083711F0083549F474D0F3010881008334
:106E600070D000E3F301008322C00F3601F5F30177
:106E700000810033E1F000E302933F0118C008E70E
:106E8000602E05E2702E462C502EF2010081002368
:106E900071F001E040D0F9CF0FEFC00ED01E0BE92A
:106EA000602E05E2702E0EE9402E05E2502E4201C2
:106EB00086189708A814B9041CF480E090E007C075
:106EC00052D0A818B90810E0A01AB10AC5010A8169
:106ED000002321F401C063D00197EAF70981002360
:106EE00039F055D004C053D0F30101913F015AD07D
:106EF0000FEF800E901EBAF70A81002309F437CEF7
:106F000001970AF434CE4BD0FBCF10E00C871D87DD
:106F10001E871F870895400E00E0501E08954C857F
:106F20005D856E857F858C019D010C944632A08322
:106F3000B18308958D919D91A083B183A0E0B0E0CD
:106F400008950FEF600E701E089580FBF701A08179
:106F5000B1810895F701A081B1810D911D91A083A8
:106F6000B183F80108950981002311F001E008952B
:106F700000E00895F60100810895F60100810053B4
:106F80000A300895F60101916F010883089528855C
:106F90003985089501E0C00E00E0D01E08952885CF
:106FA000398500E2EA85FB8509950B811C810F5F1D
:106FB0001F4F0B831C8308950E940735C801D90118
:106FC0001A013F7740E856E968E17BE40E94A53466
:106FD00038F416D0B38300E010E020E030E00DC0BC
:106FE0003B2F0E94D8320E94CB320AD03383A801B3
:106FF000B9018C019D010E946E33E4E00C941835B8
:10700000F10100831183228308950E94FB34C8019B
:10701000D901BF7741E050E060E87FE33B2F0E9459
:107020008D3470F440E00E94833429F40BED1FE0AE
:1070300029E43FE350C0CC24DD24EE24FF241CC00F
:107040000BEDC02E0FE0D02E09E4E02EF72E40E02D
:107050007FEB082F48D02801390140E050E060E87C
:107060007FE38C019D013FD0A801B901820193010A
:107070000E940434C801D901AC01BD018C019D01FD
:107080002DD02801390144E25FEF6BE27CEB26D082
:1070900048E854E466EA7EE328D048E150EC6FE328
:1070A00070E423D045EB1CD0480159014AEE54EB63
:1070B00066E870E48201930118D046EB11D0A80174
:1070C000B901840195010E940434AC01BD0106D0D0
:1070D000A601B70108D0E0E10C940C350C948B3379
:1070E0005DEF68E670E40C942A33FDDFA201B30182
:1070F000F5CF20E006D0E9F70895259102D0E9F711
:1071000008952D9301501040202F212B089588ECD5
:1071100093E7FC0105911491FC013296A591B4917D
:10712000FC01349625913491422F432B19F0F9013B
:10713000E4DF01C0DEDF069613E7843D910748F3E4
:10714000089540E00C94A4380E9403352897802FBE
:10715000B32F442E40E050E060E070E00E948D3498
:1071600010F401E001C000E0000F400EBF7743E8DB
:1071700059EF62E27FE3082F3B2F80D076D041E0C9
:107180005CEF6FE777E40E94A53488F5AE010E94BA
:10719000DC376BD0042D10E06BD0488159816A81B7
:1071A0007B8172D0088319832A833B83AE014C5FB5
:1071B0005F4F2A0140E050E060E87EE35FD0A2012B
:1071C0000E94DC3740E050E060E870E40C811D81F3
:1071D0002E813F8153D0A801B901088119812A81EC
:1071E0003B810E946E330E94D832402E0CC00E9418
:1071F000D832602E3DD0A801B9018C019D0133D059
:10720000460C03E0402240FA3EF4AC01BD0100E030
:1072100010E020E83FE327D002E0401608F0B05825
:107220008C019D0129D0280139014BEF57ED6EE10A
:1072300079E324D045E656E269E97BEB21D048E5C5
:1072400054E363EA7DE31CD041EE5DE565E27FEB4C
:1072500017D04BED5FE069EC7FE316D00DD0289698
:10726000E8E00C9414350E946E33C801D9010895EA
:1072700020E030E00C94D632AC01BD010C948B338D
:1072800003D0A201B301FACF0C942A331B2F6A2F2B
:10729000F901A081B181AD014F5F5F4F4083518300
:1072A0000C93A62FB12F0895BA93AA9324970A831B
:1072B0001B8389019E012A5F3F4F28833983BE01CA
:1072C000AE014E5F5F4F26E439E30E94A63520E011
:1072D000AA81BB812C932496A991B99108950E940B
:1072E000FF3422974801590141E050E060E070E02E
:1072F0000E948D3498F440E00E94833429F400E029
:1073000010E020E030E04EC001E2EFEAF9E2008355
:1073100051830FEF1FEF2FE73FE744C0AE010E94FC
:107320009431C801D90145EC53E062E47FE30E9447
:107330002A334AE151E562E17FE33BD0A801B9017C
:107340008C019D013BD0402E088100FF14C00A959E
:107350002DD0802F43EF54E065EB7FE3042D0E9496
:107360008B3337FB220F331F380F3695279537F9AC
:10737000C801D9010BC01AD0842D912FD90137FB38
:10738000AA0FBB1FB00FB695A795B7F940E050E024
:1073900060E87EE38C019D010CD0AC01BD0184014D
:1073A00095010CD02296ECE00C94103542E00C9440
:1073B000C0310E948B332801390108950E940434A2
:1073C000A201B3010C942A337B042421D473120448
:1073D0009F2500004E6F726D6100547572626F00E0
:1073E0005472657368004F6666004F6E004F6E2BD7
:1073F000004F6C640044796E00442B53007664693E
:10740000200056444920005376646900535644498D
:10741000002D20504C454153452057414954202DC3
:107420002000202020202020203C3E202020202042
:10743000202000204C6F772042617474657279209F
:10744000212121002045524153494E4720454550B6
:10745000524F4D212000202A726164696F646F6D64
:107460002E6F72672A20004B504F54342D474149EC
:107470004E2D53364D20202563200050726F663DFF
:1074800025642000466163746F727920736574749B
:10749000696E67730020202053657474696E67738A
:1074A000202020202000553D256420493D256420D2
:1074B000456D3D2564202020004D3D256420413D43
:1074C00025642047623D25642025642A2564200028
:1074D0005458202564487A2025646D4120200052AC
:1074E000582025646D56202020200025642A25641C
:1074F0005F257320002020205475726E20636F6911
:107500006C21003C202564206D56203E00436F69AD
:107510006C20626C3F2059657320272B27002020A8
:10752000202020202020200020256425644625647A
:10753000256300256476256420002B253032645BAA
:10754000002D253032645B005D20532564256446A0
:1075500025642563002564762564002020202020F2
:107560002F2020202020202020202000202020202C
:107570002020205050202020202020200025642082
:1075800020202020200050726F66696C652020202A
:107590002020202020200054623D25642E256456A2
:1075A000202055623D25642E2564562000426174DA
:1075B0007465727920202020203C25643E002B2514
:1075C00064202020202D2E2E2E2E2E2E2E2E2B000F
:1075D000436F6E74722E2020202020202020202037
:1075E000200025646D412020202020202020202004
:1075F0002020202000282564292E2E2E20002A4617
:107600007265715F545820256C64487A20002A46C0
:10761000657272697465202000202025642563202E
:10762000200025646D412020200025632D2E2E2E64
:107630002E2E2E2E2B00506F7765722E20202020AC
:10764000202020202020002A2564202A25642000D4
:107650002D2E2E2E2E2E2E2E2E2B004761696E20C3
:1076600020202020202020202020200025646D566E
:107670002020202020200020413D256420202000C3
:107680002A436F696C20626C2E20663D2564256359
:107690002020002564202020202000485046202063
:1076A00020202020202020202020200047726F75DD
:1076B0006E6420626C2E2000534C2E2573200056E1
:1076C0006F6C756D65202020202020202020200058
:1076D0002564746F6E6520200025732D2E2E2E2EAE
:1076E0002B00426565707320202020202020202060
:1076F00020200025732564202D2E2E2E2E2E2E2E9A
:107700002E2B00496E642B41752020202020202044
:10771000202020002573202D2E2E2E2E2E2E2E2EB4
:107720002B004D6F64652020202020202020202069
:107730002020200038363432302F30313233343587
:10774000363738530047726F756E6420626C2E4571
:1077500072726F72210047726F756E6420626C2EB8
:10776000202D4F4B2D20002020202A2A2A2025645E
:10777000202A2A2A202020200020202028253032DC
:1077800064293C253032643E202020202000202027
:107790002020202020202020202020202020002009
:1077A000204E6F204665727269746521202020008A
:1077B0002054616B652046657272697465212020D2
:1077C0000020202020204572726F7221202020206E
:1077D00020002020202020204F4B2120202020206E
:1077E0002020002020202020206C6F6E6720202089
:1077F00020202020009001303132333435363738A4
:107800003941424344454600286E756C6C20706FC8
:10781000696E746572290030313233343536373849
:107820003961626364656600464C4F4154533F20A2
:1078300077726F6E6720666F726D61747465722007
:0F784000696E7374616C6C656421003F3F3F009B
:0400000300000000F9
:00000001FF
